:020000040000FA
:06000000E4EF33F01200F2
:0600080004EF08F01200F5
:060018000CEF08F01200DD
:06100000E4EF33F01200E2
:06100800B1EF2BF0120015
:06101800BAEF2BF01200FC
:06102A0002000068000056
:10103000B600000021000000F2670000F000000090
:041040000E0000009E
:0C104400D9CFE6FFE1CFD9FFFB0EDB5057
:1010500029E10201E351EA6A000FE96E010EEA227A
:101060003C0EEF6EE329EA6A000FE96E010EEA22F8
:10107000FE0EDBCFEFFF020EE325EA6A000FE96EFA
:10108000010EEA22FD0EDBCFEFFF030EE325EA6A35
:10109000000FE96E010EEA22FC0EDBCFEFFF040E1B
:1010A000E3273BD00201E351EA6A000FE96E010E2B
:1010B000EA223C0EEF6EE329EA6A000FE96E010EA8
:1010C000EA22FE0EDBCFEFFF020EE325EA6A000FF5
:1010D000E96E010EEA22FD0EDBCFEFFF030EE325E2
:1010E000EA6A000FE96E010EEA22FC0EDBCFEFFF89
:1010F000040EE325EA6A000FE96E010EEA22FB0EF8
:10110000DBCFEFFF050EE325EA6A000FE96E010E63
:10111000EA223A0EEF6E060EE327E552E7CFD9FF3B
:101120001200D9CFE6FFE1CFD9FFFE0EDB50410818
:1011300020E1FD0EDB50350A18E0060A13E0010A33
:101140000EE0030A09E0010A04E00001CA0EB86FCC
:101150000FD0010EC26E0CD0050EC26E09D0090E62
:10116000C26E06D00D0EC26E03D0110EC26E00D03C
:101170000FD0FE0EDB5042080BE1FD0EDB50320AB1
:1011800004E00001CA0EB86F03D0210EC26E00D079
:10119000E552E7CFD9FF1200D9CFE6FFE1CFD9FF63
:1011A000FE0EDBCFE9FFEA6AE9BEEA68AB0EE9268C
:1011B000000EEA22EF50690A1DE00C0A18E0010A4D
:1011C00013E0070A0EE0010A09E0030A04E0000147
:1011D000CA0EB86F12D0010EC26E0FD0050EC26ECD
:1011E0000CD0090EC26E09D00D0EC26E06D0110EC3
:1011F000C26E03D0210EC26E00D0E552E7CFD9FFF8
:101200001200D9CFE6FFE1CFD9FFE652DF6A060E22
:10121000DF24EA6ABB0FE96E020EEA22EF50E66EA7
:10122000DF50EA6AAB0FE96E000EEA22E552E750A2
:10123000EF6EDFCFE6FFB0DFE552DF2A060EDF24D8
:10124000EA6ABB0FE96E020EEA22EF50290803E0BA
:10125000070EDF5CDCE3060EDF24EA6ABB0FE96EF3
:10126000020EEA22EF5029080CE1070EDF5C09E2CA
:10127000DF50EA6AAB0FE96E000EEA22290EEF6E2C
:1012800003D00001CC0EB86FE552E552E7CFD9FF8D
:101290001200D9CFE6FFE1CFD9FF030EE126FD0E04
:1012A000DB500F0BDF6EFD0EDB380F0B0F0BE76E05
:1012B000010EE7CFDBFFFD0EDBCF14F0FE0EDBCF20
:1012C00015F015C014F0156A0F0E1414E76E020E17
:1012D000E7CFDBFFDF50090805E2370EDF2402010C
:1012E000F46F04D0300EDF240201F46F010EDB50E6
:1012F000090805E2010EDB50370FF56F04D0010E2F
:10130000DB50300FF56F020EDB50090805E2020ECC
:10131000DB50370FF66F04D0020EDB50300FF66F44
:10132000FB0EDBCFE9FFEA6AE9BEEA687F0EE92639
:10133000020EEA22FC0EDBCFEFFFFB0EDB28E96E8C
:10134000EA6AE9BEEA687F0EE926020EEA22300E5A
:10135000EF6EFB0EDB50020FE96EEA6AE9BEEA6847
:101360007F0EE926020EEA22F6C2EFFFFB0EDB50EB
:10137000030FE96EEA6AE9BEEA687F0EE926020E0B
:10138000EA22F5C2EFFFFB0EDB50040FE96EEA6ABA
:10139000E9BEEA687F0EE926020EEA22F4C2EFFFF8
:1013A000FB0EDB50050FE96EEA6AE9BEEA687F0EC4
:1013B000E926020EEA227C0EEF6E030EE15C02E2E9
:1013C000E16AE552E16EE552E7CFD9FF1200D9CFCD
:1013D000E6FFE1CFD9FFFE0EDB50410828E1780E91
:1013E000E66EE66E8050200B01E0010E300FE66ED7
:1013F000780EE66E8050080B01E0010E300FE66EAD
:101400008050040B01E0010E300FE66E8050020B9D
:1014100001E0010E300FE66E8050010B300FE66EDA
:10142000B9EC26F0146E080EE15E145056D0FE0E94
:10143000DB50420828E1780EE66EE66E8150200B04
:1014400001E0010E300FE66E8150100B01E0010E3D
:10145000300FE66E780EE66E8150040B01E0010E4F
:10146000300FE66E8150020B01E0010E300FE66E88
:101470008150010B300FE66EB9EC26F0146E080EA9
:10148000E15E14502AD0FE0EDB50430826E1825064
:10149000800B01E0010E300FE66E8250400B01E040
:1014A000010E300FE66E780EE66EE66EE66E825046
:1014B000040B01E0010E300FE66E8250020B01E0DA
:1014C000010E300FE66E8250010B300FE66EB9EC64
:1014D00026F0146E080EE15E1450E552E7CFD9FFF6
:1014E0001200D9CFE6FFE1CFD9FFFE0EDB50410855
:1014F00001E0EED0FD0EDB50350A01E1C1D0010A5A
:1015000001E1A5D0070A01E17BD0010A52E0030AFC
:1015100029E0010A01E0DBD0FC0EDB50300802E1DB
:1015200080901FD0FC0EDB50310802E1808019D082
:10153000FC0EDB50690807E19280C1500E0802E3FF
:101540000F0EC16E0ED0FC0EDB506F0803E19290BF
:10155000809007D0FC0EDB50610803E192800E0EF4
:10156000C16EB5D0FC0EDB50300802E1809220D075
:10157000FC0EDB50310802E180821AD0FC0EDB50F9
:10158000690807E19282C1500D0802E30E0EC16E98
:101590000FD0FC0EDB506F0803E19292809208D0CE
:1015A000FC0EDB50610804E1030E92120D0EC16EB9
:1015B0008ED0FC0EDB50300802E1809420D0FC0E6F
:1015C000DB50310802E180841AD0FC0EDB50690840
:1015D00007E19284C1500C0802E30D0EC16E0FD0DA
:1015E000FC0EDB506F0803E19294809408D0FC0E4F
:1015F000DB50610804E1070E92120C0EC16E67D039
:10160000FC0EDB50300802E1809620D0FC0EDB504F
:10161000310802E180861AD0FC0EDB50690807E130
:101620009286C1500B0802E30C0EC16E0FD0FC0E67
:10163000DB506F0803E19296809608D0FC0EDB50D9
:10164000610804E10F0E92120B0EC16E40D0FC0E29
:10165000DB50300802E1809812D0FC0EDB503108DC
:1016600002E180880CD0FC0EDB50690802E1928810
:1016700006D0FC0EDB506F0802E19298809827D0CC
:10168000FC0EDB50300802E1809A20D0FC0EDB50CB
:10169000310802E1808A1AD0FC0EDB50690807E1AC
:1016A000928AC1500A0802E30B0EC16E0FD0FC0EE5
:1016B000DB506F0803E1929A809A08D0FC0EDB5051
:1016C000610804E12F0E92120A0EC16E00D082D181
:1016D000FE0EDB50420801E0EED0FD0EDB50370A73
:1016E00001E1CFD0010A01E1B3D0030A01E197D0B3
:1016F000010A01E17BD0070A60E0010A37E0030A32
:101700001CE0010A01E0D6D0FC0EDB50300802E1FB
:10171000819012D0FC0EDB50310802E181800CD0A8
:10172000FC0EDB50690802E1938006D0FC0EDB5012
:101730006F0802E193908190BDD0FC0EDB50300821
:1017400002E1819212D0FC0EDB50310802E181826D
:101750000CD0FC0EDB50690802E1938206D0FC0E2F
:10176000DB506F0802E193928192A4D0FC0EDB5013
:10177000300802E1819420D0FC0EDB50310802E1F8
:1017800081841AD0FC0EDB50690807E19384C150B4
:10179000060802E30A0EC16E0FD0FC0EDB506F0884
:1017A00003E19394819408D0FC0EDB50610804E1BE
:1017B00092689384060EC16E7DD0FC0EDB5030081B
:1017C00002E1819612D0FC0EDB50310802E18186E5
:1017D0000CD0FC0EDB50690802E1938606D0FC0EAB
:1017E000DB506F0802E19396819664D0FC0EDB50CB
:1017F000300802E1819812D0FC0EDB50310802E182
:1018000081880CD0FC0EDB50690802E1938806D079
:10181000FC0EDB506F0802E1939881984BD0FC0ED0
:10182000DB50300802E1819A12D0FC0EDB50310807
:1018300002E1818A0CD0FC0EDB50690802E1938A38
:1018400006D0FC0EDB506F0802E1939A819A32D0E9
:10185000FC0EDB50300802E1819C12D0FC0EDB5004
:10186000310802E1818C0CD0FC0EDB50690802E1EA
:10187000938C06D0FC0EDB506F0802E1939C819C98
:1018800019D0FC0EDB50300802E1819E12D0FC0E14
:10189000DB50310802E1818E0CD0FC0EDB50690870
:1018A00002E1938E06D0FC0EDB506F0802E1939E9E
:1018B000819E00D08FD0FE0EDB50430801E08AD01D
:1018C000FD0EDB50370A6DE0010A52E0040A37E0F2
:1018D000030A1CE0010A01E07DD0FC0EDB50300859
:1018E00002E1829012D0FC0EDB50310802E18280CE
:1018F0000CD0FC0EDB50690802E1948006D0FC0E8F
:10190000DB506F0802E19490829064D0FC0EDB50B3
:10191000300802E1829212D0FC0EDB50310802E165
:1019200082820CD0FC0EDB50690802E1948206D062
:10193000FC0EDB506F0802E1949282924BD0FC0EB9
:10194000DB50300802E1829412D0FC0EDB503108EB
:1019500002E182840CD0FC0EDB50690802E1948421
:1019600006D0FC0EDB506F0802E19494829432D0D2
:10197000FC0EDB50300802E1829C12D0FC0EDB50E2
:10198000310802E1828C0CD0FC0EDB50690802E1C8
:10199000948C06D0FC0EDB506F0802E1949C829C74
:1019A00019D0FC0EDB50300802E1829E12D0FC0EF2
:1019B000DB50310802E1828E0CD0FC0EDB5069084E
:1019C00002E1948E06D0FC0EDB506F0802E1949E7B
:1019D000829E00D00001C60501E1C188E552E7CF33
:1019E000D9FF1200D9CFE6FFE1CFD9FF020EE126E1
:1019F000FE0EDB500F0BDF6EFE0EDB380F0B0F0BF6
:101A0000E76E010EE7CFDBFFDF50090805E2370E76
:101A1000DF240201F46F04D0300EDF240201F46FE2
:101A2000010EDB50090805E2010EDB50370FF56FA0
:101A300004D0010EDB50300FF56FFC0EDBCFE9FF59
:101A4000EA6AE9BEEA687F0EE926020EEA22FD0E86
:101A5000DBCFEFFFFC0EDB28E96EEA6AE9BEEA683D
:101A60007F0EE926020EEA22780EEF6EFC0EDB50A6
:101A7000020FE96EEA6AE9BEEA687F0EE926020E05
:101A8000EA22780EEF6EFC0EDB50030FE96EEA6A75
:101A9000E9BEEA687F0EE926020EEA22F5C2EFFFF0
:101AA000FC0EDB50040FE96EEA6AE9BEEA687F0EBD
:101AB000E926020EEA22F4C2EFFFFC0EDB50050F0E
:101AC000E96EEA6AE9BEEA687F0EE926020EEA22BA
:101AD0007C0EEF6E020EE15C02E2E16AE552E16E1D
:101AE000E552E7CFD9FF1200D9CFE6FFE1CFD9FF0A
:101AF000FD0EDB50650810E1FE0EDB50320A07E0F8
:101B0000030A01E008D094940C0EBD6E04D09492A8
:101B10000C0EBA6E00D011D0FD0EDB5064080DE142
:101B2000FE0EDB50320A06E0030A01E006D0BD6A71
:101B3000948403D0BA6A948200D0E552E7CFD9FFEB
:101B40001200D9CFE6FFE1CFD9FFCB50146E156A52
:101B5000166A176A142A000E15221622172214C0BC
:101B600006F015C007F016C008F017C009F0FA0E0D
:101B7000DBCF0BF0FB0EDBCF0CF0FC0EDBCF0DF060
:101B8000FD0EDBCF0EF038EC32F002C006F003C0E1
:101B900007F004C008F005C009F00B6A010E0C6ED6
:101BA0000D6A0E6AEDEC30F0FA0E06C0DBFFFB0E9C
:101BB00007C0DBFFFC0E08C0DBFFFD0E09C0DBFF2A
:101BC000FE0EDB50320A0EE0030A01E016D0FA0ED8
:101BD000DBCFE6FFFB0EDBCFE6FF9FEC32F0E552FA
:101BE000E5520BD0FA0EDBCFE6FFFB0EDBCFE6FFB4
:101BF00070EC32F0E552E55200D0E552E7CFD9FF64
:101C00001200D9CFE6FFE1CFD9FFFD0EDBCF14F0F4
:101C1000FE0EDBCF15F0D890155004E62F0E145CA5
:101C2000000E15581FE3E00E086E2E0E096EFD0E15
:101C3000DBCF0DF0FE0EDBCF0EF09AEC30F008C0DB
:101C400014F009C015F01406000E155AFD0E14C04C
:101C5000DBFFFE0E15C0DBFF040EE66EA3EC33F0D7
:101C6000E55275D0FD0EDBCF14F0FE0EDBCF15F084
:101C7000D890155004E60C0E145C000E15582CE399
:101C8000FD0EDBCF16F0FE0EDBCF17F0173404E2AB
:101C900016502E08000E17541FE3B80E086E0B0ED8
:101CA000096EFD0EDBCF0DF0FE0EDBCF0EF09AECD1
:101CB00030F008C014F009C015F01406000E155AD3
:101CC000FD0E14C0DBFFFE0E15C0DBFF050EE66E39
:101CD000A3EC33F0E5523BD0FD0EDBCF14F0FE0E4B
:101CE000DBCF15F0D890155004E6030E145C000EFF
:101CF00015582CE3FD0EDBCF16F0FE0EDBCF17F0F0
:101D0000173404E216500B08000E17541FE3EE0EB2
:101D1000086E020E096EFD0EDBCF0DF0FE0EDBCF5E
:101D20000EF09AEC30F008C014F009C015F014065B
:101D3000000E155AFD0E14C0DBFFFE0E15C0DBFFB2
:101D4000060EE66EA3EC33F0E55201D0CB6AFD0E31
:101D5000DB50CB6EE552E7CFD9FF1200D9CFE6FFBB
:101D6000E1CFD9FFFE0EDB50380A3EE00F0A36E025
:101D7000010A2EE0030A26E0010A1EE0070A16E027
:101D8000010A0EE0030A06E0010A01E033D0F5EC97
:101D900033F030D0100EE66E87EC33F0E5522AD0E7
:101DA000110EE66E87EC33F0E55224D0120EE66E8B
:101DB00087EC33F0E5521ED0130EE66E87EC33F05D
:101DC000E55218D0140EE66E87EC33F0E55212D0CF
:101DD000150EE66E87EC33F0E5520CD0160EE66E6B
:101DE00087EC33F0E55206D0170EE66E87EC33F041
:101DF000E55200D0E552E7CFD9FF1200D9CFE6FF78
:101E0000E1CFD9FF060EE126DE6ADE6ADE6ADD6A10
:101E1000DD52DD52040EDB6A050EDB6AFD0EDBCF00
:101E200014F0FE0EDBCF15F0166A176A15AE02D05D
:101E30001668176814C0DFFF010E15C0DBFF020E25
:101E400016C0DBFF030E17C0DBFFFC0EDB506D0876
:101E500001E0AFD10001AA97FD0EDBCF17F0FE0E17
:101E6000DBCF18F0196A18BE1968600E146EEA0EFE
:101E7000156E166A14C007F015C008F016C009F0F8
:101E800017C00CF018C00DF019C00EF0C0EC30F007
:101E900007C0CAF008C0CBF0FD0EDBCF14F0FE0E79
:101EA000DBCF15F0153404E21450F408010E15547C
:101EB00041E2FD0EDBCF16F0FE0EDBCF17F017343C
:101EC00004E21650E708030E175434E3170EE66ECB
:101ED00087EC33F0E552D9CFE9FFDACFEAFFEECF56
:101EE00006F0EECF07F0EECF08F0EFCF09F01B0EB3
:101EF0000B6EB70E0C6E0D6A0E6A38EC32F002C033
:101F000006F003C007F004C008F005C009F0E80EB1
:101F10000B6E030E0C6E0D6A0E6ACEEC32F006C02C
:101F2000DEFF07C0DEFF08C0DEFF09C0DDFFDD52B7
:101F3000DD5209D1FD0EDBCF14F0FE0EDBCF15F024
:101F4000153404E214506408000E155442E2FD0EEC
:101F5000DBCF16F0FE0EDBCF17F0173404E216507D
:101F6000F408010E175435E3160EE66E87EC33F0D5
:101F7000E552D9CFE9FFDACFEAFFEECF06F0EECF98
:101F800007F0EECF08F0EFCF09F0360E0B6E6E0EB5
:101F90000C6E010E0D6E0E6A38EC32F002C006F0C7
:101FA00003C007F004C008F005C009F0E80E0B6E8E
:101FB000030E0C6E0D6A0E6ACEEC32F006C0DEFF28
:101FC00007C0DEFF08C0DEFF09C0DDFFDD52DD52C5
:101FD000BAD0FD0EDBCF14F0FE0EDBCF15F01534BA
:101FE00004E214503208000E155431E2FD0EDBCF2E
:101FF00016F0FE0EDBCF17F0173404E2165064081B
:10200000000E175424E3140EE66E87EC33F0E5520D
:10201000D9CFE9FFDACFEAFFEECF06F0EECF07F037
:10202000EECF08F0EFCF09F0770E0B6E010E0C6EBD
:102030000D6A0E6A38EC32F002C0DEFF03C0DEFF2C
:1020400004C0DEFF05C0DDFFDD52DD527CD0FD0E99
:10205000DBCF14F0FE0EDBCF15F0153404E2145084
:102060000A08000E155431E2FD0EDBCF16F0FE0E0D
:10207000DBCF17F0173404E216503208000E175465
:1020800024E3130EE66E87EC33F0E552D9CFE9FF77
:10209000DACFEAFFEECF06F0EECF07F0EECF08F092
:1020A000EFCF09F0EE0E0B6E020E0C6E0D6A0E6A8B
:1020B00038EC32F002C0DEFF03C0DEFF04C0DEFFFA
:1020C00005C0DDFFDD52DD523ED0FD0EDBCF14F04A
:1020D000FE0EDBCF15F0D890155004E6010E145C0F
:1020E000000E155830E3FD0EDBCF16F0FE0EDBCFF1
:1020F00017F0173404E216500A08000E175423E3B1
:10210000100EE66E87EC33F0E552D9CFE9FFDACF57
:10211000EAFFEECF06F0EECF07F0EECF08F0EFCFFC
:1021200009F0700E0B6E170E0C6E0D6A0E6A38EC0D
:1021300032F002C0DEFF03C0DEFF04C0DEFF05C0D8
:10214000DDFFDD52DD52176A186A010E196EDFCF0E
:102150001AF0DBCF1BF01C6A1BBE1C681A50175C00
:10216000146E1B501858156E1C501958166E190E07
:102170001426000E15221622040E14C0DBFF050ED5
:1021800015C0DBFFF294040EDBCFE6FF050EDBCFBC
:10219000E6FF6BEC33F0E552E552040EDBCF14F0B2
:1021A000050EDBCF15F014C0F3FF15C0F4FF9ED071
:1021B0009DD0FC0EDB50750801E095D00001AA8788
:1021C0000001E80ECC6F030ECD6FFD0EDBCF17F0D4
:1021D000FE0EDBCF18F0196A18BE1968600E146E77
:1021E000EA0E156E166A14C007F015C008F016C086
:1021F00009F017C00CF018C00DF019C00EF0C0ECBB
:1022000030F007C0CAF008C0CBF0FD0EDBCF14F0F1
:10221000FE0EDBCF15F0D890155004E6010E145CCD
:10222000000E15582FE3FD0EDBCF16F0FE0EDBCFB0
:1022300017F0173404E21650E708030E175422E390
:10224000100EE66E87EC33F0E552D9CFE9FFDACF16
:10225000EAFFEECF06F0EECF07F0EECF08F0EFCFBB
:1022600009F0060E0B6E0C6A0D6A0E6A38EC32F03D
:1022700002C0DEFF03C0DEFF04C0DEFF05C0DDFFDD
:10228000DD52DD52176A186A010E196EDFCF1AF09F
:10229000DBCF1BF01C6A1BBE1C681A50175C146E47
:1022A0001B501858156E1C501958166E040E14C089
:1022B000DBFF050E15C0DBFFF294040EDBCFE6FF5B
:1022C000050EDBCFE6FF6BEC33F0E552E552040E72
:1022D000DBCF14F0050EDBCF15F014C0F3FF15C0F3
:1022E000F4FF04D003D00001CB0EB86F060EE15C02
:1022F00002E2E16AE552E16EE552E7CFD9FF120052
:10230000D9CFE6FFE1CFD9FFFE0EDB50340A1EE045
:10231000070A16E0010A0EE0030A06E0010A01E0DE
:102320001BD0F2EC33F018D04D0EE66EF2EC32F02A
:10233000E55212D05D0EE66EF2EC32F0E5520CD0B2
:102340006D0EE66EF2EC32F0E55206D07D0EE66ED2
:10235000F2EC32F0E55200D0E552E7CFD9FF12009F
:10236000D9CFE6FFE1CFD9FF060EE126DE6ADE6AAD
:10237000DE6ADD6ADD52DD52040EDB6A050EDB6AC1
:10238000FD0EDBCF14F0FE0EDBCF15F0166A176AD8
:1023900015AE02D01668176814C0DFFF010E15C015
:1023A000DBFF020E16C0DBFF030E17C0DBFFFC0EC7
:1023B000DB506D0801E029D1FD0EDBCF14F0FE0EDD
:1023C000DBCF15F0153404E214501408000E155438
:1023D00031E2FD0EDBCF16F0FE0EDBCF17F0173427
:1023E00004E216502808000E175424E37D0EE66E12
:1023F000F2EC32F0E552D9CFE9FFDACFEAFFEECFC7
:1024000006F0EECF07F0EECF08F0EFCF09F0DC0ECC
:102410000B6E050E0C6E0D6A0E6A38EC32F002C0BF
:10242000DEFF03C0DEFF04C0DEFF05C0DDFFDD52BE
:10243000DD52BAD0FD0EDBCF14F0FE0EDBCF15F06F
:10244000153404E214500A08000E155431E2FD0E52
:10245000DBCF16F0FE0EDBCF17F0173404E2165078
:102460001408000E175424E36D0EE66EF2EC32F001
:10247000E552D9CFE9FFDACFEAFFEECF06F0EECF93
:1024800007F0EECF08F0EFCF09F0B80E0B6E0B0E91
:102490000C6E0D6A0E6A38EC32F002C0DEFF03C02B
:1024A000DEFF04C0DEFF05C0DDFFDD52DD527CD063
:1024B000FD0EDBCF14F0FE0EDBCF15F0153404E279
:1024C00014500508000E155431E2FD0EDBCF16F056
:1024D000FE0EDBCF17F0173404E216500A08000E88
:1024E000175424E35D0EE66EF2EC32F0E552D9CFDC
:1024F000E9FFDACFEAFFEECF06F0EECF07F0EECF3E
:1025000008F0EFCF09F0700E0B6E170E0C6E0D6A0F
:102510000E6A38EC32F002C0DEFF03C0DEFF04C0FA
:10252000DEFF05C0DDFFDD52DD523ED0FD0EDBCF0C
:1025300014F0FE0EDBCF15F0D890155004E6010E16
:10254000145C000E155830E3FD0EDBCF16F0FE0EC6
:10255000DBCF17F0173404E216500508000E1754AD
:1025600023E34D0EE66EF2EC32F0E552D9CFE9FFEF
:10257000DACFEAFFEECF06F0EECF07F0EECF08F0AD
:10258000EFCF09F0E00E0B6E2E0E0C6E0D6A0E6A88
:1025900038EC32F002C0DEFF03C0DEFF04C0DEFF15
:1025A00005C0DDFFDD52DD52176A186A010E196E93
:1025B000DFCF1AF0DBCF1BF01C6A1BBE1C681A5061
:1025C000175C146E1B501858156E1C501958166E57
:1025D000040E14C0DBFF050E15C0DBFF9E90040E39
:1025E000DBCFE6FF050EDBCFE6FF4FEC33F0E55225
:1025F000E552040EDBCF14F0050EDBCF15F014C04E
:10260000F3FF15C0F4FF76D075D0FC0EDB507508D3
:102610006EE1FD0EDBCF14F0FE0EDBCF15F0D8908F
:10262000155004E6010E145C000E15582FE3FD0E44
:10263000DBCF16F0FE0EDBCF17F0173404E2165096
:10264000E708030E175422E34D0EE66EF2EC32F06B
:10265000E552D9CFE9FFDACFEAFFEECF06F0EECFB1
:1026600007F0EECF08F0EFCF09F00C0E0B6E0C6AFE
:102670000D6A0E6A38EC32F002C0DEFF03C0DEFFE6
:1026800004C0DEFF05C0DDFFDD52DD52176A186AA7
:10269000010E196EDFCF1AF0DBCF1BF01C6A1BBED8
:1026A0001C681A50175C146E1B501858156E1C507D
:1026B0001958166E040E14C0DBFF050E15C0DBFFA3
:1026C0009E90040EDBCFE6FF050EDBCFE6FF4FEC5E
:1026D00033F0E552E552040EDBCF14F0050EDBCFEC
:1026E00015F014C0F3FF15C0F4FF04D003D00001AF
:1026F000CB0EB86F060EE15C02E2E16AE552E16ED4
:10270000E552E7CFD9FF1200D9CFE6FFE1CFD9FFDD
:10271000040EE126DF6A010EDB6A020EDB6A030E9D
:10272000DB6A5A0E0201BC5D1DE14D0EBD5D19E173
:10273000440EBE5D16E1310EE66E760EE66E320E8A
:10274000E66E310EE66E500EE66E430EE66E690ED4
:10275000E66E3A0EE66EB9EC26F0146E080EE15EF7
:102760001450AAD04D0EBC5D1BE1440EBD5D08E1C6
:10277000490EBE5D05E10F0EC16E926893680FD0E1
:10278000410EBD5D0CE14E0EBE5D09E19268040E86
:10279000936E010EC26E060EC16EBF0EC06E8CD05F
:1027A000440EBC5D01E088D0500EBD5D2BE1410EB2
:1027B000BE5D28E1780EE66EE66E8050200B01E0EB
:1027C000010E300FE66E780EE66E8050080B01E0C9
:1027D000010E300FE66E8050040B01E0010E300F49
:1027E000E66E8050020B01E0010E300FE66E805065
:1027F000010B300FE66EB9EC26F0146E080EE15EA8
:1028000014505AD0500EBD5D2BE1420EBE5D28E142
:10281000780EE66EE66E8150200B01E0010E300F5F
:10282000E66E8150100B01E0010E300FE66E780E5F
:10283000E66E8150040B01E0010E300FE66E815010
:10284000020B01E0010E300FE66E8150010B300FDC
:10285000E66EB9EC26F0146E080EE15E14502CD032
:10286000500EBD5D29E1430EBE5D26E18250800B16
:1028700001E0010E300FE66E8250400B01E0010EC8
:10288000300FE66E780EE66EE66EE66E8250040B52
:1028900001E0010E300FE66E8250020B01E0010EE6
:1028A000300FE66E8250010B300FE66EB9EC26F069
:1028B000146E080EE15E1450020E0001B85D02E1D4
:1028C0000201BF6B040EE15C02E2E16AE552E16ED7
:1028D000E552E7CFD9FF1200D9CFE6FFE1CFD9FF0C
:1028E000E652F250800B01E0010EDF6EF29EA69ED2
:1028F000A69CA684FE0EDB50A96EFD0EDB50A86ED2
:10290000550EA76EAA0EA76EA682A6B2FED7A694F3
:10291000DF50E8B0F28EE8A0F29EE552E552E7CF34
:10292000D9FF1200D9CFE6FFE1CFD9FFA69CA69E22
:10293000FE0EDB50A96EA680A85000D0E552E7CF6E
:10294000D9FF1200D9CFE6FFE1CFD9FFE652FB0E47
:10295000DB50F66EFC0EDB50F76EFD0EDB50F86EB2
:10296000E00EF616DF6ADFCF14F03F0EE76E1418A4
:10297000E8AE02D0143403D0E750D880145412E3E8
:102980000900DFCF14F0156A14BE1568F90EDB508C
:102990001424E96EFA0EDB501520EA6EF5CFEFFF36
:1029A000DF2AE1D7E552E552E7CFD9FF1200D9CFB0
:1029B000E6FFE1CFD9FFE652A6B2FED7F29CF29E27
:1029C000FD0EDB50F86EFC0EDB50F76EFB0EDB509D
:1029D000F66EE00EF616A68EA69CA684A688550E68
:1029E000A76EAA0EA76EA6820000F90EDBCF14F028
:1029F000FA0EDBCF15F015C014F0156A1450EA6E0C
:102A0000FF0EE76EF90EDBCF14F0FA0EDBCF15F0F8
:102A1000E7501416156A1450E96E0A00200EDF6E96
:102A2000DF5005E0EE50F56E0F00DF06F9D7A68EF9
:102A3000A69CA684550EA76EAA0EA76EA6820000BD
:102A4000200EDF6EDF5005E0EE50F56E0F00DF0662
:102A5000F9D7A68EA69CA684550EA76EAA0EA76EC1
:102A6000A6820000A694F28EF28CE552E552E7CFE2
:102A7000D9FF1200550EA76EAA0EA76EA682A6B2A7
:102A8000FED7A6941200D9CFE6FFE1CFD9FFF29C82
:102A9000F29EFD0EDB50F86EFC0EDB50F76EFB0E67
:102AA000DB50F66E0001FE6B0E0E0001FE5D17E2BC
:102AB0000001FE51E76EF90EDBCFE9FFFA0EDBCF26
:102AC000EAFFE750E926000EEA22EF50F56E0C000F
:102AD000C40EA66ECFDF09000001FE2BE5D7F28EF3
:0A2AE000F28CE552E7CFD9FF120097
:062AEA00D9CFE6FFE1CFA9
:102AF000D9FFE652A09A6A6A686A706A020EE66EA8
:102B0000E66AE66A710EE66E0F0EE66E1EEC32F0B5
:102B1000146E050EE15E1450160E6F6E9F0E6B6EF6
:102B20007B0E696EDF6ADF50146E156A0C0E145C42
:102B3000000E155810E2DF50040DF3CFE9FFF4CF7B
:102B4000EAFF000EE926040EEA22EE6AEE6AEE6A59
:102B5000EE6ADF2AE8D76D8C6E6A6D986D9C68A668
:102B600007D068960001776B7C6B7D6B7E6BF7D727
:102B70000001010E906F916F926B936B846BDF6A13
:102B8000030EDF5C26E2EA6ADF34FE0BEA36E96E0A
:102B90006D0EE926000EEA22EE6AED6AEA6ADF347B
:102BA000FE0BEA36E96E670EE926000EEA22EE6AAF
:102BB000ED6ADF50EA6A880FE96E000EEA22EF6ADA
:102BC000DF50EA6A8B0FE96E000EEA22EF6ADF2A15
:102BD000D7D70001080E6D6F040E6E6F160E706E63
:102BE0000401300E026F040E036F080E016F840E95
:102BF000006F0001616B606BE552E552E7CFD9FFD2
:102C00001200D9CFE6FFE1CFD9FFE65200016051B3
:102C100016E106D06D6A696A0001606BA19AB9D0AD
:102C20006D6A696A160E6F6E9F0E6B6E7B0E696E13
:102C30006DB602D06D86FCD70001010E606F600595
:102C400008E16DBA06D0686A696A69806988020E0F
:102C5000606F6850040B05E06950040B02E0689453
:102C6000CBD86DA202D0A19A94D06850010B08E095
:102C70006950010B05E039DF0001040E606F6890B8
:102C80006850100B05E06950100B02E0A0D868985E
:102C900068AC19D069AC0FD0010EE66EE66A000E82
:102CA000E66EE66A730EE66EE66A20EC2EF0146EAF
:102CB000060EE15E1450689C00018E5101E08E0703
:102CC0008E5101E165DB6850200B04E06950200B58
:102CD00001E064D86850020B13E06950020B10E069
:102CE000010EE66EE66A000EE66EE66AE6687F0EA4
:102CF000E66E20EC2EF0146E060EE15E14506A6A49
:102D0000040E0001E76E6019E8AE02D0E73402D08D
:102D1000E750605D02E2A19A3CD069A639D0DF6A33
:102D2000040EDF5C35E268A630D06CCF85F0000180
:102D30008551780BE842E842E842866F689685B58F
:102D400008D08651EA6A8B0FE96E000EEA22EF7016
:102D500007D08651EA6A880FE96E000EEA22EF700A
:102D6000865102E160D810D0000EE66EE66A850E4C
:102D7000E66E000EE66E720EE66EE66A20EC2EF04F
:102D8000146E060EE15E145001D002D0DF2AC8D7BF
:102D9000A19AE552E552E7CFD9FF120070A015D0F5
:102DA00063C0E9FF64C0EAFFEF5080080DE16DC029
:102DB000E9FF6EC0EAFFEF50840806E163C0E9FF57
:102DC00064C0EAFF8C0EEF6E7090689A12006984FE
:102DD00068986D820001010E846F000EE66EE66A4F
:102DE000E66EE66A750EE66EE66A20EC2EF0146E6C
:102DF000060EE15E145012000001846B000EE66EB8
:102E0000E66AE66EE66A740EE66EE66A20EC2EF07E
:102E1000146E060EE15E14506D92699468A402D09F
:102E20006894FCD71200D9CFE6FFE1CFD9FFE65274
:102E300000012D0E8E6FFD0E851553E17E0E85155A
:102E4000E8407F0B040DF3CF63F0F4CF64F0000E85
:102E50006327040E642363C065F064C066F0657583
:102E600063C0E9FF64C0EAFFEF503C0BE842E84270
:102E70000D0835E1DF6A080EDF5C23E263C0E9FF7D
:102E800064C0EAFF020EE926000EEA22EE50EFCF00
:102E9000EAFFE96EEF50E66EDF50EA6A300FE96E46
:102EA000040EEA22E552E750EF6E63C0E9FF64C00A
:102EB000EAFF020EE926000EEA22EE2AEF22DF2ABE
:102EC000DAD763C0E9FF64C0EAFF020EE926000E0C
:102ED000EA22300EEE6E040EED6E0DD801D03AD817
:102EE00005D0FD0E8515040801E15AD8E552E552DA
:102EF000E7CFD9FF12000001736B8F6B926B936B5E
:102F0000876B746B6DC0E9FF6EC0EAFFEF9E6D7555
:102F10006DC0E9FF6EC0EAFFEF9E6D7565C0E9FF09
:102F200066C0EAFFEF9E776B786B796B7C6B7D6B8D
:102F30007E6B90D8000EE66EE66AE66EE66A030ED9
:102F4000E66EE66A20EC2EF0146E060EE15E14507A
:102F50001AEF1BF0020E0001745D03E1DDEC1BF0C3
:102F60001ED0746B87511AE165C0E9FF66C0EAFFA5
:102F7000EE52080EEF6E65C0E9FF66C0EAFF020E72
:102F8000E926000EEA22300EEE6E040EED6E65C0EC
:102F9000E9FF66C0EAFF8C0EEF6E01D0876B12006E
:102FA000D9CFE6FFE1CFD9FFE6526DC0E9FF6EC091
:102FB000EAFFEF50400B01E0010EDF6E00016D757E
:102FC000080E605D09E132C46EFF6E5003E0100E22
:102FD000606F02D0040E606F740528E16DC0E9FFD8
:102FE0006EC0EAFF020EE926000EEA22380EEE6EEF
:102FF000040EED6E80DB020E0001735D07E16DC013
:10300000E9FF6EC0EAFF840EEF6E0FD0DF5007E1DC
:103010006DC0E9FF6EC0EAFFC80EEF6E06D06DC04E
:10302000E9FF6EC0EAFF880EEF6E0FD07CAF0CD0C8
:103030007F51801107E005D080C0FAFF00017F5169
:10304000F96EFADF00017C9F746BE552E552E7CF21
:10305000D9FF120004013051600BE842E842E84217
:10306000E842E842000901E059D031510C0A55E02C
:103070000B0A44E00C0A36E0010A27E00B0A23E0C1
:10308000020A21E0030A1DE0080A11E0010A0CE02F
:103090000F0A08E0030A01E040D00001778F080E14
:1030A000606F3CD006DA3AD07DEC1CF037D00001DE
:1030B000610E756F000E766F7781010E786F778FD6
:1030C0002DD057DA2BD02BD829D034510001756F71
:1030D000766B620E7527000E76237781010E786F6E
:1030E000778F1CD00001778F04013451EA6A620F98
:1030F000E96E000EEA2232C4EFFF10D0000EE66E39
:10310000E66AE66EE66A020EE66EE66A20EC2EF0ED
:10311000146E060EE15E145001D000D01200D9CF1B
:10312000E6FFE1CFD9FF030EE1260401320510E1ED
:1031300030511F0B00090CE10001778F030E0401D1
:10314000315D04E10001010E836F02D00001836B49
:103150000401325101E012D130511F0B020801E08D
:103160000DD134510F0B000901E108D134510F0B7F
:10317000020801E203D1200E0001605D01E0FED0F3
:10318000778F040134BF1AD034510F0BE96EEA6A0D
:10319000D890E936EA36670EE926000EEA22EECF2D
:1031A000DEFFEDCFDDFF34510F0BEA6A8B0FE96EC6
:1031B000000EEA22020EEFCFDBFF19D034510F0BC5
:1031C000E96EEA6AD890E936EA366D0EE926000E15
:1031D000EA22EECFDEFFEDCFDDFF34510F0BEA6ABE
:1031E000880FE96E000EEA22020EEFCFDBFFD95006
:1031F000020FE96EDACFEAFFEF50010B03E1000E98
:10320000DF9401D0DF8434BF10D034510F0BE96E4E
:10321000EA6AD890E936EA36670EE926000EEA2215
:10322000DECFEEFFDDCFEDFF0FD034510F0BE96E97
:10323000EA6AD890E936EA366D0EE926000EEA22EF
:10324000DECFEEFFDDCFEDFF030E315D23E1DECFFC
:10325000E9FFDDCFEAFFEF50800B13E034BF09D068
:1032600034510F0BEA6A8B0FE96E000EEA22EF82EF
:1032700008D034510F0BEA6A880FE96E000EEA227B
:10328000EF82840E146EDECFE9FFDDCFEAFF14502B
:10329000EF1274D0DF74DECFE9FFDDCFEAFFEF502D
:1032A000800B1BE0DECFE9FFDDCFEAFFEF9EDECF34
:1032B000E9FFDDCFEAFFEF8C020EE66EE66ADECFB5
:1032C000E6FFDDCFE6FF050EE66EE66A20EC2EF0A7
:1032D000146E060EE15E145005D0DECFE9FFDDCF9F
:1032E000EAFFEF8CDF74D950020FE96EDACFEAFF04
:1032F000EF50020B0EE1DECFE9FFDDCFEAFFEF502A
:10330000800B34E0DECFE9FFDDCFEAFFEF50040BA6
:103310002DE1040134BF09D034510F0BEA6A8B0F41
:10332000E96E000EEA22EF9208D034510F0BEA6AE0
:10333000880FE96E000EEA22EF923B0E146EDECF8C
:10334000E9FFDDCFEAFF1450EF16020EE66EE66AE3
:10335000DECFE6FFDDCFE6FF050EE66EE66A20EC87
:103360002EF0146E060EE15E145008D03B0E146E63
:10337000DECFE9FFDDCFEAFF1450EF16030EE15C6C
:1033800002E2E16AE552E16EE552E7CFD9FF1200B1
:10339000000190514DE1010E906F915149E1010EF4
:1033A000916F020E745D0DE16DC0E9FF6EC0EAFF22
:1033B000EE52EF6A6DC0E9FF6EC0EAFFC80EEF6E15
:1033C00037D0740535E1876B63C0E9FF64C0EAFF5D
:1033D000EE52080EEF6E63C0E9FF64C0EAFF020E12
:1033E000E926000EEA22300EEE6E040EED6E63C08A
:1033F000E9FF64C0EAFF840EEF6E010E876F65C0BF
:10340000E9FF66C0EAFFEE52080EEF6E65C0E9FF05
:1034100066C0EAFF020EE926000EEA22300EEE6ECA
:10342000040EED6E65C0E9FF66C0EAFF800EEF6E28
:1034300012000001926B936B020E745D1AE165C07D
:10344000E9FF66C0EAFFEE52080EEF6E65C0E9FFC5
:1034500066C0EAFF020EE926000EEA22380EEE6E82
:10346000040EED6E65C0E9FF66C0EAFFC80EEF6EA0
:103470001FD078510401365D00017951040137599C
:1034800004E236C478F037C479F035D96DC0E9FF6D
:103490006EC0EAFF020EE926000EEA22380EEE6E3A
:1034A000040EED6E6DC0E9FF6EC0EAFFC80EEF6E50
:1034B0001200800E0401305D5BE10001C00E776FE9
:1034C00004013351030A34E0010A0EE0030A03E069
:1034D0000001776B4DD000017E0E756F620E766F26
:1034E000120E786F796B44D03251F66EF76AD8902D
:1034F000F636F7363F0EF626630EF7220900F5CFB3
:1035000075F00A00F5CF76F0020E0001F76A752516
:10351000F66E7651F7220800F5CF78F0030EF76AC1
:103520007525F66E7651F7220800F5CF79F020D098
:10353000030E325D1AE23251F66EF76AD890F63613
:10354000F736410EF626630EF7220900F5CF75F027
:103550000A00F5CF76F075C0F6FF76C0F7FF0800D9
:10356000F5500001786F796B02D00001776B00D0C5
:103570001200D9CFE6FFE1CFD9FF020EE126040108
:10358000386B396B30511F0B020A12E0030A0DE051
:10359000010A01E03BD00001778F0401388100016E
:1035A000830502E10401388331D00001778F2ED0EA
:1035B0000001778F040134BF10D034510F0BE96E36
:1035C000EA6AD890E936EA36670EE926000EEA2262
:1035D000EECFDEFFEDCFDDFF0FD034510F0BE96EE4
:1035E000EA6AD890E936EA366D0EE926000EEA223C
:1035F000EECFDEFFEDCFDDFFDECFE9FFDDCFEAFF6F
:10360000EF50040B02E0010E386F00D0000177AFDD
:1036100007D0380E756F040E766F7781020E786FC3
:10362000020EE15C02E2E16AE552E16EE552E7CFAB
:10363000D9FF12006D98000177BF2BD07CAF09D065
:10364000020E746F935101E1F4DE0001916B906BF7
:103650001FD065C0E9FF66C0EAFFEE52080EEF6EAC
:1036600065C0E9FF66C0EAFF020EE926000EEA2205
:10367000300EEE6E040EED6E65C0E9FF66C0EAFF27
:103680008C0EEF6E6DC0E9FF6EC0EAFF840EEF6E28
:1036900031D0040130AF0DD00001010E746F925192
:1036A00001E1C7DE0001916B906B8F5101E170DE8B
:1036B00021D00001020E746F65C0E9FF66C0EAFF09
:1036C000EE52080EEF6E65C0E9FF66C0EAFF020E1B
:1036D000E926000EEA22300EEE6E040EED6E65C095
:1036E000E9FF66C0EAFF840EEF6E916B906B8F511D
:1036F00001E14EDE1200D9CFE6FFE1CFD9FFE6525D
:10370000080EDF6E0001785D000E79590BE278C07B
:10371000DFFF735103E1010E736F04D0730502E103
:10372000020E736FDF50146E156A1450785D786F57
:1037300015507959796F6DC0E9FF6EC0EAFFEE52FE
:10374000DFCFEFFF380E816F040E826F77B119D093
:10375000DF5016E075C0F6FF76C0F7FF752B000E40
:1037600076230800F550E66E81C0E9FF82C0EAFFCB
:10377000812B000E8223E552E750EF6EDF06E8D77B
:1037800017D0DF5015E075C0E9FF76C0EAFF752B52
:10379000000E7623EF50E66E81C0E9FF82C0EAFF9B
:1037A000812B000E8223E552E750EF6EDF06E9D74A
:1037B000E552E552E7CFD9FF1200D9CFE6FFE1CFBE
:1037C000D9FF020EE12663C0E9FF64C0EAFFEE52B2
:1037D000EFCFDFFFDFCF14F0145000017D5D000E4E
:1037E0007E5902E27DC0DFFFDF50146E156A14506F
:1037F0007D5D7D6F15507E597E6F010EDB6ADF5057
:10380000F36E010EDBCFF4FFF350F45C16E2010E11
:10381000DB50EA6A380FE96E040EEA22EF50E66EDA
:103820007AC0E9FF7BC0EAFF7A2B000E7B23E552CA
:10383000E750EF6E010EDB2AE2D7000ED8807D55EF
:10384000000E7E5528E265C0E9FF66C0EAFFEE5231
:10385000080EEF6E65C0E9FF66C0EAFF020EE926BA
:10386000000EEA22380EEE6E040EED6E63C0E9FF24
:1038700064C0EAFFEF50400B07E165C0E9FF66C096
:10388000EAFFC80EEF6E06D065C0E9FF66C0EAFF2A
:10389000880EEF6E28D065C0E9FF66C0EAFFEE52E1
:1038A000080EEF6E65C0E9FF66C0EAFF020EE9266A
:1038B000000EEA22300EEE6E040EED6E65C0E9FFDA
:1038C00066C0EAFF840EEF6E7F51801107E005D0DD
:1038D00080C0FAFF00017F51F96EFADF00017C9F82
:1038E0008F5101E155DD020EE15C02E2E16AE55231
:1038F000E16EE552E7CFD9FF1200D9CFE6FFE1CF65
:10390000D9FFE6520001778F020EE66EE66AE66A9C
:10391000710EE66E0F0EE66E1EEC32F0146E050EA2
:10392000E15E1450DF6ADF50146E156A0C0E145CF1
:10393000000E155810E2DF50040DF3CFE9FFF4CF6D
:10394000EAFF000EE926040EEA22EE6AEE6AEE6A4B
:10395000EE6ADF2AE8D76D8C010EE66EE66AE66A4B
:10396000620EE66E000EE66E1EEC32F0146E050E70
:10397000E15E14506D9C0001080E6D6F040E6E6FB9
:10398000000E636F040E646F63C065F064C066F080
:1039900032C461F0615103E1100E606F13D0010E6B
:1039A000E66EE66A610EE66E000EE66E010EE66EEB
:1039B000E66A20EC2EF0146E060EE15E1450000153
:1039C000200E606FE552E552E7CFD9FF1200D9CF44
:1039D000E6FFE1CFD9FF020EE126000EDE6E040EF7
:1039E000DD6EFD0EDB50E824166EFE0EDB50040D7E
:1039F000F3501624040DF3CF14F0F4CF15F0D9CF03
:103A0000E9FFDACFEAFF1450EE261550ED22DECFA3
:103A1000E9FFDDCFEAFFEF9EFD0EDB500FE1FE0E6A
:103A2000EA6ADB34FE0BEA36E96E670EE926000E21
:103A3000EA22DECFEEFFDDCFEDFF0ED0FE0EEA6A0A
:103A4000DB34FE0BEA36E96E6D0EE926000EEA2243
:103A5000DECFEEFFDDCFEDFFDECFE9FFDDCFEAFF0A
:103A6000EF9CDECFE9FFDDCFEAFF040EE926000E72
:103A7000EA22EF8C020EE15C02E2E16AE552E16EBD
:103A8000E552E7CFD9FF1200D9CFE6FFE1CFD9FF4A
:103A9000020EE126FD0EDBA407D0E66AFE0EDBCFA8
:103AA000E6FF95DFE552E552FD0EDBA208D0010EE0
:103AB000E66EFE0EDBCFE6FF8ADFE552E552FE0E34
:103AC000DB50156A700F146E0F0E152214C0DEFF46
:103AD00015C0DDFFDECFE9FFDDCFEAFFFD0EDBCF56
:103AE000EFFF020EE15C02E2E16AE552E16EE552AF
:103AF000E7CFD9FF1200D9CFE6FFE1CFD9FF020E01
:103B0000E126FE0EDB5020E165C0E9FF66C0EAFF5A
:103B1000EE52080EEF6E65C0E9FF66C0EAFF020EC6
:103B2000E926000EEA22300EEE6E040EED6E65C040
:103B3000E9FF66C0EAFF8C0EEF6E6DC0E9FF6EC054
:103B4000EAFF840EEF6E3DD0FD0EDB50E824166ECA
:103B5000FE0EDB50040DF3501624040DF3CF14F0C9
:103B6000F4CF15F0000E1426040E152214C0DEFF4B
:103B700015C0DDFF840E146EDECFE9FFDDCFEAFF56
:103B80001450EF12FD0EDB50E824166EFE0EDB50D3
:103B9000040DF3501624010F040DF3CF14F0F4CFED
:103BA00015F0000E1426040E152214C0DEFF15C0F9
:103BB000DDFF840E146EDECFE9FFDDCFEAFF145087
:103BC000EF12020EE15C02E2E16AE552E16EE552BB
:103BD000E7CFD9FF1200D9CFE6FFE1CFD9FF020E20
:103BE000E126FD0EDB500FE0FE0EEA6ADB34FE0B31
:103BF000EA36E96E6D0EE926000EEA22EECFDEFF10
:103C0000EDCFDDFF0ED0FE0EEA6ADB34FE0BEA36A6
:103C1000E96E670EE926000EEA22EECFDEFFEDCF59
:103C2000DDFFD9CFE9FFDACFEAFFEE50ED1003E177
:103C3000F36AF46A49D0DECFE9FFDDCFEAFF020E76
:103C4000E926000EEA22FB0EDBCFEEFFFC0EDBCFF7
:103C5000EDFFDECFE9FFDDCFEAFFEE52FA0EDBCF5C
:103C6000EFFF400E146EDECFE9FFDDCFEAFF145008
:103C7000EF16880E146EDECFE9FFDDCFEAFF145099
:103C8000EF12FD0EDB500CE0FE0EEA6ADB34FE0B99
:103C9000EA36E96E6D0EE926000EEA22EF740BD0CB
:103CA000FE0EEA6ADB34FE0BEA36E96E670EE926A1
:103CB000000EEA22EF74DECF14F0DDCF15F014C051
:103CC000F3FF15C0F4FF00D0020EE15C02E2E16AEE
:103CD000E552E16EE552E7CFD9FF1200D9CFE6FFFA
:103CE000E1CFD9FF6DA84ED0FE0EEA6ADB34FE0BA1
:103CF000EA36E96E6D0EE926000EEA22EE50EFCFAD
:103D0000EAFFE96E400EEE16EE6AEE6AEE6AFE0E0D
:103D1000EA6ADB34FE0BEA36E96E6D0EE926000E28
:103D2000EA22EE50EFCFEAFFE96EEE7CFE0EEA6A81
:103D3000DB34FE0BEA36E96E6D0EE926000EEA2250
:103D4000EF74400E146EFE0EEA6ADB34FE0BEA36A8
:103D5000E96E6D0EE926000EEA22EE50EFCFEAFF83
:103D6000E96E1450EF16FE0EEA6ADB34FE0BEA36FB
:103D7000E96E6D0EE926000EEA22EE50EFCFEAFF63
:0C3D8000E96EEF7CE552E7CFD9FF12009E
:043D8C009EAC96D083
:103D90009E9CC3CFC1F0C4CFC2F00001F95102E034
:103DA0006BEC25F00001A8B525D0C1C0E6FFC2C06C
:103DB000E6FF7EEC27F0E552E5520201300E7F6F00
:103DC000806F0201F7250201816F300E0201F62596
:103DD0000201826F300E0201F5250201836F300E61
:103DE0000201F4250201846F3E0E856F0001030E6F
:103DF000B86F64D00001C329EA6AAB0FE96E000E08
:103E0000EA22EF50290803E0050EC35D32E3C3C088
:103E1000B6F0060EB603F3500001F0250001B76FAF
:103E2000B7C0E6FFB651EA6AAB0FE96E000EEA22B0
:103E3000EF50E66EC1C0E6FFC2C0E6FF49EC09F0F4
:103E4000E552E552E552E552050E0001B725EA6A52
:103E50007F0FE96E020EEA223E0EEF6EE66ACCECB0
:103E600008F0E5520001C36B030EB86F0001A99181
:103E700025D0C32BC3C0E6FFCCEC08F0E552C282CC
:103E80000001C305B66F060EB603F3500001F0251E
:103E90000001B76FB7C0E6FFB651EA6AAB0FE96E33
:103EA000000EEA22EF50E66EC1C0E6FFC2C0E6FF98
:103EB00049EC09F0E552E552E552E5521200D9CF3E
:103EC000E6FFE1CFD9FF070EE126DF6A010EDB6ACC
:103ED000020EDB6A0001AAA11AD0050EDB6A060EEB
:103EE000DB6A050EDB2A060E01E3DB2A000ED65C38
:103EF0000EE3FF0ED75C0BE1050EDBCF14F0060ED0
:103F0000DBCF15F0E80E145C030E1558EAE3F2A4BB
:103F1000ACD0F294030ED6CFDBFF040ED7CFDBFF7D
:103F2000DBCF16F016C017F0166A030EDB50000147
:103F30001610146E17C015F0010E14C0DBFF020E30
:103F400015C0DBFFD950010FE96EDACFEAFF00019F
:103F5000D351EE26D451ED22010EDBCF14F0020E28
:103F6000DBCF15F015C014F0156A1450D76E010E92
:103F7000DB50D66E0001AAA178D08A7A0201540ED5
:103F8000BC6FBD6F300EBE6F720EBF6F0001AAA373
:103F90000FD0010EDF6EA9810001F06B0001BC6B38
:103FA000C36AC46AE66ACCEC08F0E5529E9CC28201
:103FB0000001AAA52CD0E66A410EE66E8050E66E9E
:103FC000F2EC0CF0E552E552E552060EE66E420EBA
:103FD000E66E8150E66EF2EC0CF0E552E552E552E9
:103FE0000C0EE66E430EE66E8250E66EF2EC0CF0BE
:103FF000E552E552E5520001120EF06FDF5007E185
:10400000F06B02013E0E906F0001030EB86F0001CD
:10401000C851C91118E00001AAB705D00001C807AE
:10402000000EC95B0FD00001CC51CD1104E0CC07CC
:10403000000ECD5B07D0E80ECC6F030ECD6FC80726
:10404000000EC95B07D0C851C91104E10001AA9153
:10405000A9918A9A0001A951040B07E00001C751F8
:1040600004E1040EC76FB96BBA6B070EE15C02E2A4
:10407000E16AE552E16EE552E7CFD9FF1200000197
:10408000A895A891A893410E0201BD5D03E0420EE0
:10409000BD5D1EE1630EBF5D09E1BEC2E6FFBDC2AC
:1040A000E6FF91EC08F0E552E55211D0720EBF5DCB
:1040B0000EE10001630EB86FB96BBA6BBEC2E6FFCA
:1040C000BDC2E6FF91EC08F0E552E552C2824CD049
:1040D000430EBD5D2EE14D0EBE5D2BE1650EBF5D55
:1040E0000FE13A0EC05D0CE10001A885AA83000132
:1040F000C36B01EC09F0E66ACCEC08F0E55218D08D
:10410000640EBF5D03E10001AA9312D0720EBF5D81
:104110000FE10001A8850001F06B0001C36B630E85
:10412000B86FB96BBA6BE66ACCEC08F0E552C282A4
:104130001BD0560EBD5D12E1500EBE5D0FE1650E47
:10414000BF5D05E1C1880001010EC66F06D0640E97
:10415000BF5D03E1C1980001C66B06D0540EBD5D82
:1041600003E1560EBE5D00E1120012001200500E77
:104170000201BD5D32E1770EBF5D26E10001B66B45
:10418000080EB65D20E2060EB625EA6ABB0FE96EA0
:10419000020EEA22EF50780813E0060EB625EA6A0E
:1041A000BB0FE96E020EEA22EF50E66E300EB62526
:1041B000E66EBEC2E6FF71EC0AF0E552E552E5524A
:1041C0000001B62BDDD708D0720EBF5D05E1BEC27F
:1041D000E6FFE7EC09F0E552BCD0430EBD5D3BE1E4
:1041E0004D0EBE5D38E1650EBF5D03E10001AA859D
:1041F00031D0640EBF5D03E10001AA952BD0720E91
:10420000BF5D28E1E66A410EE66E8050E66EF2EC94
:104210000CF0E552E552E552060EE66E420EE66EF1
:104220008150E66EF2EC0CF0E552E552E5520C0ED0
:10423000E66E430EE66E8250E66EF2EC0CF0E5524E
:10424000E552E55202013E0E906F0001F06B000155
:10425000030EB86F7ED0550EBD5D10E1420EBE5DFF
:1042600005E1650EBF5D02E1F19E07D0420EBE5D25
:1042700004E1640EBF5D01E1F18E6BD04D0EBD5DBA
:1042800068E1650EBF5D03E0640EBF5D09E1BFC27A
:10429000E6FFBEC2E6FF74EC0DF0E552E55259D0E0
:1042A000660EBF5D1FE16B0EC45D1CE1C3C2E6FF7D
:1042B000C2C2E6FFC1C2E6FF300EE66EE66EDFEC7C
:1042C00026F0146E050EE15E1450F3CFBFF0F4CF6C
:1042D000C0F0BFC0E6FFC0C0E6FF01EC0EF0E55243
:1042E000E55237D0720EBF5D34E1C4C2E6FFC3C2EF
:1042F000E6FFC2C2E6FFC1C2E6FF300EE66EDFECAB
:1043000026F0146E050EE15E1450F3CFBFF0F4CF2B
:10431000C0F00001000ED880BF55000EC05503E26A
:10432000BF2B000EC023BFC014F0C0C015F0166A2A
:10433000176A14C0E6FF15C0E6FF16C0E6FF17C0F7
:10434000E6FFBEC2E6FFA1EC0DF0186E050EE15EC1
:1043500018501200BFC2E6FFBEC2E6FFBDC2E6FFB4
:1043600071EC0AF0E552E552E5521200300E0201FE
:10437000BE5D01E0B2D0700EBF5D06E1C1C2E6FFD6
:10438000AEEC0EF0E552A8D0640EBF5D09E100016D
:10439000AA91300EE66EAEEC0EF0E5528A9A9CD0F1
:1043A000710EBF5D34E1C5C2E6FFC4C2E6FFC3C201
:1043B000E6FFC2C2E6FFC1C2E6FFDFEC26F0146EE4
:1043C000050EE15E1450F3CFBFF0F4CFC0F0176AD2
:1043D000186A010E196EBFC01AF0C0C01BF01C6A2B
:1043E0001A50175C146E1B501858156E1C50195833
:1043F000166E14C0D3F015C0D4F0F294D3C0E6FF0B
:10440000D4C0E6FF6BEC33F0E552E55265D0740E94
:10441000BF5D31E1C3C2E6FFC2C2E6FFC1C2E6FF33
:10442000300EE66EE66EDFEC26F0146E050EE15EF1
:104430001450F3CFBFF0F4CFC0F0C4C2E6FFBFC04A
:10444000E6FFC0C0E6FFFEEC0EF0E552E552E55295
:10445000F3CFD3F0F4CFD4F000010A0ED880BF55CB
:10446000000EC05505E30001A9850001C76B02D00D
:104470000001A99531D0630EBF5D25E1C4C2E6FFFE
:10448000C3C2E6FFC2C2E6FFC1C2E6FF300EE66E5F
:10449000DFEC26F0146E050EE15E1450F3CFBFF092
:1044A000F4CFC0F00001BF51C0110CE0BFC0CAF092
:1044B000C0C0CBF0010ECA5F000ECB5BCAC0C8F013
:1044C000CBC0C9F009D0720EBF5D06E10001AA8120
:1044D000CAC0C8F0CBC0C9F071D0310EBE5D6EE16C
:1044E000700EBF5D06E1C1C2E6FF80EC11F0E5523F
:1044F00065D0640EBF5D06E1300EE66E80EC11F013
:10450000E5525CD0720EBF5D34E1C5C2E6FFC4C2A5
:10451000E6FFC3C2E6FFC2C2E6FFC1C2E6FFDFECB0
:1045200026F0146E050EE15E1450F3CFBFF0F4CF09
:10453000C0F0176A186A010E196EBFC01AF0C0C029
:104540001BF01C6A1A50175C146E1B501858156E1D
:104550001C501958166E14C0D5F015C0D6F09E9098
:10456000D5C0E6FFD6C0E6FF4FEC33F0E552E5528A
:1045700025D0740EBF5D22E1C3C2E6FFC2C2E6FFD2
:10458000C1C2E6FF300EE66EE66EDFEC26F0146E7A
:10459000050EE15E1450F3CFBFF0F4CFC0F0C4C2FB
:1045A000E6FFBFC0E6FFC0C0E6FFB0EC11F0E55289
:1045B000E552E552F3CFD5F0F4CFD6F012004D0E10
:1045C0000201BD5D1DE1440EBE5D1AE1720EBF5DCC
:1045D00017E1310EE66E760EE66E410EE66E320E95
:1045E000E66E310EE66E500EE66E430EE66E690E16
:1045F000E66EB9EC26F0146E080EE15E145084D01D
:10460000460EBD5D1BE1570EBE5D18E1720EBF5D2B
:1046100015E1300EE66E350EE66E310EE66E300EAA
:10462000E66EE66EE66E310EE66E300EE66EB9ECC4
:1046300026F0146E080EE15E145066D0490EBD5D82
:104640001BE1440EBE5D18E1720EBF5D15E1EFDAAD
:10465000B2C0E6FFB3C0E6FFB4C0E6FFB5C0E6FFF8
:10466000300EE66EE66EE66EE66EB9EC26F0146E7F
:10467000080EE15E145048D0440EBD5D10E1300ECE
:10468000BF5D146E300EBE5D0A0DF35014240001A0
:10469000F96F0001BD6BBE6B010EB86F35D0530EC4
:1046A000BD5D14E1490EBE5D11E1770EBF5D0EE107
:1046B0009268CF0E936E94680F0EC16E806A816A05
:1046C000826A0001B86B0001F46B1ED0520EBD5D12
:1046D0001BE14F0EBE5D18E1520EBF5D15E1C4C275
:1046E000E6FFC3C2E6FFC2C2E6FFC1C2E6FFB7EC07
:1046F0002AF0E552E552E552E552F3CFC1F0F4CF8E
:10470000C2F00001010EB86F12000001B86BC56B5A
:104710000001F46B0001F96B0001AA91AA93AA951C
:10472000A891A893A895A991A9950001C76B12001B
:104730000201E551EA6A3F0FE96E020EEA22EF50EC
:10474000280852E10001F16B0201E551EA6A3F0FCE
:10475000E96E020EEA22EF50E66E0001F151EA6ABC
:10476000BB0FE96E020EEA22E552E750EF6E02013E
:10477000E551EA6A3F0FE96E020EEA22EF6A000194
:10478000F12B0201E52B0201E4510201E55D0DE28E
:10479000E551EA6A3F0FE96E020EEA22EF5029085E
:1047A00004E0140E0001F15DCFE30201E551EA6A75
:1047B0003F0FE96E020EEA22EF50E66E0001F15162
:1047C000EA6ABB0FE96E020EEA22E552E750EF6E8D
:1047D000F151EA6ABB0FE96E020EEA22EF50290896
:1047E00003E10001010EF46F12000001F60555E12E
:1047F0000001F75152E10001F66B0001F16B00017D
:10480000B66BB651EA6ACF0FE96E020EEA22EF509C
:1048100028080AE00001F2510001B65D05E2140E1D
:10482000B65D02E2B62BEDD7B651EA6ACF0FE96E5C
:10483000020EEA22EF50E66E0001F151EA6ABB0F68
:10484000E96E020EEA22E552E750EF6E0001B65122
:10485000EA6ACF0FE96E020EEA22EF6A0001F12B3D
:104860000001B62BB605EA6ACF0FE96E020EEA2206
:10487000EF50290808E00001F2510001B65D03E2A3
:10488000140EB65DD1E30001F2510001B65D02E302
:104890000001F26B0001010EF46F0001F4052FE13D
:1048A0000001B8512CE10201BC515A0A1AE00E0A6B
:1048B00016E0060A12E0020A0EE0160A0AE0020AF0
:1048C00006E0050A01E00FD03FEC20F00CD04DDCF3
:1048D0000AD04CDC08D04BDC06D03CDD04D046DDF1
:1048E00002D06DDE00D00001B85102E184EC13F07B
:1048F0000001B85102E1010EB86F0201BB6B12005A
:104900000001B85102E1E6D070D0B8050EE1B86BF5
:104910000201E351EA6A000FE96E010EEA22230E5A
:10492000EF6EE32B0001F46B60D0020EB85D03E084
:10493000030EB85D5AE1C75101E0C707020EB85D2A
:1049400003E1080EB76F05D0030EB85D02E13C0E1F
:10495000B76FB86BBFC2E6FFBEC2E6FFBDC2E6FFDF
:10496000BCC2E6FF22EC08F0E552E552E552E55202
:104970000001B66BB62BB651EA6A7F0FE96E020EE4
:10498000EA22EF503E0803E0B751B65DF3E3B651BB
:10499000E66EE66A7F0EE66E020EE66E0201E351F7
:1049A000156A000F146E010E152214C0E6FF15C023
:1049B000E6FFF3EC31F0166E060EE15E16500001D4
:1049C000B651EA6A7F0FE96E020EEA22EF6AB6512B
:1049D0000201E327E351EA6A000FE96E010EEA22C1
:1049E0003E0EEF6EE32B0001F46B630E0001B85D29
:1049F00007E00001A951010B03E10001C7510DE0DF
:104A00000001B92B000EBA23280EB95D230EBA5946
:104A100004E3B96BBA6BCD0EB86FB851146E156A5A
:104A2000153404E21450C808000E155453E2B8516E
:104A3000C16FC26BC80EC15F000EC25BC1C0E6FF92
:104A4000C2C0E6FF7EEC27F0E552E5520201E351D9
:104A5000EA6A000FE96E010EEA223C0EEF6EE329CE
:104A6000EA6A000FE96E010EEA225A0EEF6E020E9C
:104A7000E325EA6A000FE96E010EEA22450EEF6EA9
:104A8000300E0201F525E66E030E0201E325EA6A07
:104A9000000FE96E010EEA22E552E750EF6E300E8C
:104AA0000201F425E66E040E0201E325EA6A000F16
:104AB000E96E010EEA22E552E750EF6E050EE3259E
:104AC000EA6A000FE96E010EEA223E0EEF6E060E54
:104AD000E3271BDE12000001F90511E10001E80ED9
:104AE000BD5D030EBE5903E3BD6BBE6B03D0BD2B92
:104AF000000EBE23BDC0C1F0BEC0C2F021D0020E68
:104B0000F95D07E113EC33F0F3CFC1F0F4CFC2F05D
:104B100017D0030EF95D11E10001BC2B300EBC254E
:104B2000E66E0201E351EA6A000FE96E010EEA2225
:104B3000E552E750EF6EE32B03D0040EF95D00E180
:104B400012000001D2050EE1ACA2FED70201E55130
:104B5000EA6A3F0FE96E020EEA22EF50E66E41EC80
:104B60002CF0E5521200D9CFE6FFE1CFD9FF040EB9
:104B7000E1260001C16BC26BFF0EE66E010EE66E10
:104B8000C1C014F0C2C015F0166A176A14C0E6FF5F
:104B900015C0E6FF16C0E6FF17C0E6FFA2EC14F052
:104BA000186E060EE15E1850FFC1DFFF010E00C255
:104BB000DBFF0001200EC16F080EC26FFF0EE66E14
:104BC000010EE66EC1C014F0C2C015F0166A176A75
:104BD00014C0E6FF15C0E6FF16C0E6FF17C0E6FFEB
:104BE000A2EC14F0186E060EE15E1850020EFFC122
:104BF000DBFF030E00C2DBFFDF500DE1010EDB50D7
:104C00000AE1020EDB50ED0806E1030EDB5010084E
:104C100002E103D002D08A8AFFD7040EE15C02E2EF
:104C2000E16AE552E16EE552E7CFD9FF1200D9CF34
:104C3000E6FFE1CFD9FF040EE1263F0EF86EF768DC
:104C4000FE0EF66E0800F550DF6EF6680800010EE5
:104C5000F5CFDBFF0F0EDF14E76E020EE7CFDBFFB1
:104C6000DF380F0B0F0BE76E030EE7CFDBFF020EF3
:104C7000DB50090806E2020EDB50370F0001B26F6D
:104C800005D0020EDB50300F0001B26F030EDB5077
:104C9000090806E2030EDB50370F0001B36F05D0A1
:104CA000030EDB50300F0001B36F010EDB500F0B12
:104CB000E76E020EE7CFDBFF010EDB380F0B0F0BA9
:104CC000E76E030EE7CFDBFF020EDB50090806E2BA
:104CD000020EDB50370F0001B46F05D0020EDB501F
:104CE000300F0001B46F030EDB50090806E2030E1B
:104CF000DB50370F0001B56F05D0030EDB50300FCE
:104D00000001B56F040EE15C02E2E16AE552E16E7A
:084D1000E552E7CFD9FF1200C4
:084D1800D9CFE6FFE1CFD9FF7E
:104D2000FD0EDBCFE9FFFE0EDBCFEAFFEF501DE00B
:104D3000FD0EDBCFE9FFFE0EDBCFEAFFEF50E66EA4
:104D40000201E351EA6A000FE96E010EEA22E55220
:104D5000E750EF6EE32BFD0EDBCFE9FFDB2AFE0E03
:104D6000DBCFEAFF01E3DB2ADBD7E552E7CFD9FF50
:104D70001200D9CFE6FFE1CFD9FFFE0EDBCF7FF2E5
:104D8000FD0EDBCF80F2FC0EDBCF81F2FB0EDBCF22
:104D900082F2FA0EDBCF83F2F90EDBCF84F2F80E4B
:104DA000DBCF85F2F70EDBCF86F202013E0E876F76
:104DB0000001020EB86FE552E7CFD9FF1200D9CF3C
:104DC000E6FFE1CFD9FF020EE126DE6ADD6AFE0EC4
:104DD000DBCF14F0156A14BE1568300E145E000E99
:104DE000155A100E1502F3CF15F0270E1402F350CA
:104DF0001526100E1402F3CF14F0F450152614C02B
:104E0000DEFF15C0DDFFFD0EDBCF14F0156A14BE0A
:104E10001568300E145E000E155AE80E1502F3CF19
:104E200015F0030E1402F3501526E80E1402F3CF0A
:104E300014F0F4501526D9CFE9FFDACFEAFF145069
:104E4000EE261550ED22FC0EDBCF14F0156A14BED1
:104E50001568300E145E000E155A640E1502F3CF5D
:104E600015F01402F3CF14F0F4501526D9CFE9FF52
:104E7000DACFEAFF1450EE261550ED22FB0EDBCF01
:104E800014F0156A14BE1568300E145E000E155A23
:104E90000A0E1502F3CF15F01402F3CF14F0F450FC
:104EA0001526D9CFE9FFDACFEAFF1450EE261550C8
:104EB000ED22FA0EDBCF14F0156A14BE1568300E21
:104EC000145E000E155AD9CFE9FFDACFEAFF14506D
:104ED000EE261550ED22DECF14F0DDCF15F014C014
:104EE000F3FF15C0F4FF020EE15C03E200D0E16ABB
:104EF000E552E16EE552E7CFD9FF1200D9CFE6FFC8
:104F0000E1CFD9FF0201F86BF76BF66BF56BF46B31
:104F1000D950FD0FE96EFF0EDA20EA6EEE50ED106B
:104F200001E121D3FD0EDBCF14F0FE0EDBCF15F037
:104F3000D890155004E6E80E145C030E155801E2F3
:104F400083D0FD0EDBCF14F0FE0EDBCF15F0D89032
:104F5000155004E6A00E145C0F0E155813E3040E52
:104F6000F76FFD0EDBCF14F0FE0EDBCF15F0A00EB9
:104F7000145E0F0E155AFD0E14C0DBFFFE0E15C099
:104F8000DBFF62D0FD0EDBCF14F0FE0EDBCF15F0A1
:104F9000D890155004E6B80E145C0B0E155813E3A8
:104FA000030EF76FFD0EDBCF14F0FE0EDBCF15F016
:104FB000B80E145E0B0E155AFD0E14C0DBFFFE0E6C
:104FC00015C0DBFF41D0FD0EDBCF14F0FE0EDBCFB2
:104FD00015F0D890155004E6D00E145C070E155845
:104FE00013E3020EF76FFD0EDBCF14F0FE0EDBCFE6
:104FF00015F0D00E145E070E155AFD0E14C0DBFF1F
:10500000FE0E15C0DBFF20D0FD0EDBCF14F0FE0E30
:10501000DBCF15F0D890155004E6E80E145C030EB3
:10502000155812E3010EF76FFD0EDBCF14F0FE0EE4
:10503000DBCF15F0E80E145E030E155AFD0E14C0FA
:10504000DBFFFE0E15C0DBFFFD0EDBCF14F0FE0E06
:10505000DBCF15F0D890155004E6F40E145C010E69
:10506000155801E2A5D0FD0EDBCF14F0FE0EDBCF0C
:1050700015F0D890155004E6840E145C030E1558F4
:1050800013E3090EF66FFD0EDBCF14F0FE0EDBCF3F
:1050900015F0840E145E030E155AFD0E14C0DBFFCE
:1050A000FE0E15C0DBFF83D0FD0EDBCF14F0FE0E2D
:1050B000DBCF15F0D890155004E6200E145C030EDB
:1050C000155813E3080EF66FFD0EDBCF14F0FE0E3D
:1050D000DBCF15F0200E145E030E155AFD0E14C022
:1050E000DBFFFE0E15C0DBFF62D0FD0EDBCF14F040
:1050F000FE0EDBCF15F0D890155004E6BC0E145C04
:10510000020E155813E3070EF66FFD0EDBCF14F0F9
:10511000FE0EDBCF15F0BC0E145E020E155AFD0E0E
:1051200014C0DBFFFE0E15C0DBFF41D0FD0EDBCF50
:1051300014F0FE0EDBCF15F0D890155004E6580E93
:10514000145C020E155813E3060EF66FFD0EDBCF4E
:1051500014F0FE0EDBCF15F0580E145E020E155A39
:10516000FD0E14C0DBFFFE0E15C0DBFF20D0FD0ED0
:10517000DBCF14F0FE0EDBCF15F0D890155004E60F
:10518000F40E145C010E155812E3050EF66FFD0EB9
:10519000DBCF14F0FE0EDBCF15F0F40E145E010E23
:1051A000155AFD0E14C0DBFFFE0E15C0DBFF92D0BA
:1051B000FD0EDBCF14F0FE0EDBCF15F0D8901550AE
:1051C00004E6640E145C000E155801E283D0FD0E57
:1051D000DBCF14F0FE0EDBCF15F0D890155004E6AF
:1051E000900E145C010E155813E3040EF66FFD0EBD
:1051F000DBCF14F0FE0EDBCF15F0900E145E010E27
:10520000155AFD0E14C0DBFFFE0E15C0DBFF62D089
:10521000FD0EDBCF14F0FE0EDBCF15F0D89015504D
:1052200004E62C0E145C010E155813E3030EF66F02
:10523000FD0EDBCF14F0FE0EDBCF15F02C0E145E4E
:10524000010E155AFD0E14C0DBFFFE0E15C0DBFF6C
:1052500041D0FD0EDBCF14F0FE0EDBCF15F0D89061
:10526000155004E6C80E145C000E155813E3020E28
:10527000F66FFD0EDBCF14F0FE0EDBCF15F0C80E7F
:10528000145E000E155AFD0E14C0DBFFFE0E15C095
:10529000DBFF20D0FD0EDBCF14F0FE0EDBCF15F0D0
:1052A000D890155004E6640E145C000E155812E3F5
:1052B000010EF66FFD0EDBCF14F0FE0EDBCF15F006
:1052C000640E145E000E155AFD0E14C0DBFFFE0EB8
:1052D00015C0DBFFFD0EDBCF14F0FE0EDBCF15F0AB
:1052E000D890155004E6320E145C000E155801E2F9
:1052F000A5D0FD0EDBCF14F0FE0EDBCF15F0D8905D
:10530000155004E65A0E145C000E155813E3090EEE
:10531000F56FFD0EDBCF14F0FE0EDBCF15F05A0E4D
:10532000145E000E155AFD0E14C0DBFFFE0E15C0F4
:10533000DBFF83D0FD0EDBCF14F0FE0EDBCF15F0CC
:10534000D890155004E6500E145C000E155813E367
:10535000080EF56FFD0EDBCF14F0FE0EDBCF15F05F
:10536000500E145E000E155AFD0E14C0DBFFFE0E2B
:1053700015C0DBFF62D0FD0EDBCF14F0FE0EDBCFDD
:1053800015F0D890155004E6460E145C000E155822
:1053900013E3070EF56FFD0EDBCF14F0FE0EDBCF2F
:1053A00015F0460E145E000E155AFD0E14C0DBFFFC
:1053B000FE0E15C0DBFF41D0FD0EDBCF14F0FE0E5C
:1053C000DBCF15F0D890155004E63C0E145C000EAF
:1053D000155813E3060EF56FFD0EDBCF14F0FE0E2D
:1053E000DBCF15F03C0E145E000E155AFD0E14C0F6
:1053F000DBFFFE0E15C0DBFF20D0FD0EDBCF14F06F
:10540000FE0EDBCF15F0D890155004E6320E145C7A
:10541000000E155812E3050EF56FFD0EDBCF14F0EC
:10542000FE0EDBCF15F0320E145E000E155AFD0E87
:1054300014C0DBFFFE0E15C0DBFF92D0FD0EDBCFEC
:1054400014F0FE0EDBCF15F0D890155004E60A0ECE
:10545000145C000E155801E283D0FD0EDBCF14F072
:10546000FE0EDBCF15F0D890155004E6280E145C24
:10547000000E155813E3040EF56FFD0EDBCF14F08C
:10548000FE0EDBCF15F0280E145E000E155AFD0E31
:1054900014C0DBFFFE0E15C0DBFF62D0FD0EDBCFBC
:1054A00014F0FE0EDBCF15F0D890155004E61E0E5A
:1054B000145C000E155813E3030EF56FFD0EDBCFE1
:1054C00014F0FE0EDBCF15F01E0E145E000E155A02
:1054D000FD0E14C0DBFFFE0E15C0DBFF41D0FD0E3C
:1054E000DBCF14F0FE0EDBCF15F0D890155004E69C
:1054F000140E145C000E155813E3020EF56FFD0E2A
:10550000DBCF14F0FE0EDBCF15F0140E145E000E90
:10551000155AFD0E14C0DBFFFE0E15C0DBFF20D0B8
:10552000FD0EDBCF14F0FE0EDBCF15F0D89015503A
:1055300004E60A0E145C000E155812E3010EF56F16
:10554000FD0EDBCF14F0FE0EDBCF15F00A0E145E5D
:10555000000E155AFD0E14C0DBFFFE0E15C0DBFF5A
:10556000FD0EDBCFF4F2E552E7CFD9FF1200D9CF21
:10557000E6FFE1CFD9FF0A0EE126FE0EDB50390827
:105580000EE3FE0EDB50D00F146E156A14BE1568C4
:10559000080E14C0DBFF090E15C0DBFF11D0FE0E94
:1055A000DB5039080DE2FE0EDB50C90F146E156A90
:1055B00014BE1568080E14C0DBFF090E15C0DBFF12
:1055C000086A100E096E080EDBCF0DF0090EDBCF56
:1055D0000EF021EC31F0080E06C0DBFF090E07C00B
:1055E000DBFFFD0EDB5039080EE3FD0EDB50D00F64
:1055F000146E156A14BE1568060E14C0DBFF070E84
:1056000015C0DBFF11D0FD0EDB5039080DE2FD0E99
:10561000DB50C90F146E156A14BE1568060E14C04F
:10562000DBFF070E15C0DBFF086A010E096E060ED0
:10563000DBCF0DF0070EDBCF0EF021EC31F0060EC4
:1056400006C0DBFF070E07C0DBFFFC0EDB5039088E
:105650000EE3FC0EDB50D00F146E156A14BE1568F5
:10566000040E14C0DBFF050E15C0DBFF11D0FC0ECD
:10567000DB5039080DE2FC0EDB50C90F146E156AC1
:1056800014BE1568040E14C0DBFF050E15C0DBFF49
:10569000100E086E096A040EDBCF0DF0050EDBCF8D
:1056A0000EF021EC31F0040E06C0DBFF050E07C042
:1056B000DBFFFB0EDB5039080EE3FB0EDB50D00F97
:1056C000146E156A14BE1568020E14C0DBFF030EBB
:1056D00015C0DBFF11D0FB0EDB5039080DE2FB0ECD
:1056E000DB50C90F146E156A14BE1568020E14C083
:1056F000DBFF030E15C0DBFF060EDBCF1AF0070E33
:10570000DBCF1BF0080EDB501A24186E090EDB509D
:105710001B20196E040EDB501824166E050EDB508C
:105720001920176E020EDB501624146E030EDB5088
:105730001720156E14C0DEFF15C0DDFFDECF14F09C
:10574000DDCF15F014C0F3FF15C0F4FF0A0EE15CC5
:1057500003E200D0E16AE552E16EE552E7CFD9FFFE
:02576000120035
:0E576200DACFE4FFE2CFDAFFE652E552E5CF00
:10577000DAFF1100D8CFE4FFE0CFE4FFE46EDACF28
:10578000E4FFE2CFDAFFE652E552E5CFDAFFE5507B
:10579000E5CFE0FFE5CFD8FF100011D80001A9B197
:1057A00002D001EC16F00001A9B105D00CD9F5EC3E
:1057B00023F05FEC1FF0C6EC1EF0F0D712000F0EC6
:1057C000C11202D875EF15F0D9CFE6FFE1CFD9FFAE
:1057D000E6520001D26B0001010EFA6FDF6ADF5062
:1057E000146E156AFF0E145C000E155809E2DF50A6
:1057F000EA6A000FE96E010EEA22EF6ADF2AEFD7AC
:105800000201E36BE46BE66BE76BCF0E93169268D5
:10581000936E9468C26A0F0EC16EBE0EC06E070E04
:10582000B46E806A816A826ADF6A080EDF5C09E210
:10583000DF50EA6A7F0FE96E020EEA22EF6ADF2A82
:10584000F4D785EC23F0B3EC25F0E552E552E7CF31
:10585000D9FF1200D9CFE6FFE1CFD9FFE652938AF4
:10586000939E240EAC6E900EAB6E670EAF6EB06A58
:10587000080EB86EAE50DF6EE552E552E7CFD9FFA5
:105880001200D9CFE6FFE1CFD9FFFE0EDB50AD6E9F
:10589000E552E7CFD9FF1200D9CFE6FFE1CFD9FF1C
:1058A000050EE126A00E0501001907E1860E01197B
:1058B00004E1010E021901E1035116E10001010E9C
:1058C000F36F939681966D926D6ADF6AFF0EDF5CCF
:1058D00009E2E868E85004E0E80600D000D0FAD712
:1058E000DF2AF4D700EF00F0D880000E0501005544
:1058F000C20E0155010E0255000E035501E244D0BF
:105900000001010EFA6F00C5CFF501C5D0F502C543
:10591000D1F503C5D2F5186A1B0E196EB70E1A6EB3
:105920001B6A18C006F019C007F01AC008F01BC0A7
:1059300009F0CFC50BF0D0C50CF0D1C50DF0D2C524
:105940000EF0CEEC32F006C014F007C015F008C01F
:1059500016F009C017F01406000E155A000E165A5C
:10596000000E175A010E14C0DBFF020E15C0DBFF3C
:10597000030E16C0DBFF040E17C0DBFF010EDB5069
:10598000AF6E020EDB50B06E050EE15C02E2E16A22
:10599000E552E16EE552E7CFD9FF1200D9CFE6FF1D
:1059A000E1CFD9FFE652ABA205D0AB98AE50DF6E87
:1059B000AB8802D0AE50DF6EDF5000D0E552E5522A
:1059C000E7CFD9FF1200D9CFE6FFE1CFD9FFE652EA
:1059D0000A0E0001F95D06E10B0EF96F0001010EE0
:1059E000D26F38DF0001D2510FE1200E0001E76EC7
:1059F0006019E8AE02D0E73402D0E750605D03E3FF
:105A00006D50020B01E0A6D00001FB5115E1400EE4
:105A1000E66E3F0EE66E020EE66EF7EC2EF0E552F5
:105A2000E552E5520201E46FE451000805E200018D
:105A3000010EFB6F0201E56B0001FB5111E0AC5060
:105A4000020B0EE0F4510CE10001B85109E198ECB1
:105A500023F00201E52BE451E55D02E30001FB6B5D
:105A60000001D85103E00001D20502E180EC24F0EE
:105A70000001D2052EE10001F6512BE1F45129E19C
:105A80009E50200B26E08ADFE66E0001F251EA6AA2
:105A9000CF0FE96E020EEA22E552E750EF6EF251A7
:105AA000EA6ACF0FE96E020EEA22EF50280802E1FF
:105AB000010EF56FF251EA6ACF0FE96E020EEA228B
:105AC000EF50290805E1F50503E1F56B010EF66FCE
:105AD000F22B0201E35100083BE20001C75138E11B
:105AE0000001FA0519E1F85117E10001D85114E15C
:105AF000E3C2E6FF000EE66E010EE66E58EC2FF0F4
:105B0000E552E552E5520001D20504E10001010E23
:105B1000F86F02D00201E36B0001D20519E1AC502D
:105B2000020B16E00001F751EA6A000FE96E010E60
:105B3000EA22EF50E66EA5DEE5520001F72B0201E6
:105B4000E3510001F75D04E3F76BF86B0201E36BCF
:105B5000F4EC2FF0E552E552E7CFD9FF1200000137
:105B6000FC51FD1104E1100EFC6F270EFD6FFC07C8
:105B7000000EFD5B6DA20AD0FC51FD1106E18A7892
:105B80008AA802D08A8A01D08A9A2ED00001605158
:105B900003E18A988A9A28D0600503E18A888A8A74
:105BA00023D0020E605D03E18A888A9A1DD0040E1C
:105BB000605D03E18A988A8A17D0100E605D07E164
:105BC0000001FC51FD1102E18A788A9A0DD0200E65
:105BD000605D0AE10001FC51FD1106E18A788AA8A6
:105BE00002D08A9A01D08A8A120012001200120092
:105BF00012006FEF2EF01200C2EF2EF000018305AD
:105C00001EE1000184051BE1F1DF6D920001846B50
:105C10000201100EE86F0E0EE96FE807000EE95B57
:105C2000E851E911FAE16D84080EE86F070EE96F9B
:105C3000E807000EE95BE851E911FAE16D94120002
:105C4000D9CFE6FFE1CFD9FFFD0EDBCF08F0FE0E86
:105C5000DBCF09F0050E081801E1095039E0E868CA
:105C6000081802E17F0E091831E0030E081801E15F
:105C700009502AE0020E081801E1095023E0010E44
:105C8000081801E109501CE0740E081801E10950E0
:105C900015E0750E081801E109500EE0730E0818A2
:105CA00001E1095007E0720E081801E1095001E016
:105CB00010D00FD09CDF0DD098DF0BD097DF09D02C
:105CC0009BDF07D098DF05D094DF03D091DF01D0B0
:0E5CD00000D0010E00D0E552E7CFD9FF120040
:025CDE000401BF
:105CE00030511F0B010801E04CD03051600BE842ED
:105CF000E842E842E842E842010801E042D034517B
:105D000003E0340501E03DD03151220A35E0030AB9
:105D100028E0010A17E0210A0EE0010A01E031D073
:105D20000001E80E756F000E766F080E786F796BC4
:105D30007781778F26D00001E80E756F000E766FA1
:105D4000778F1FD036C47DF037C47EF00001000E7F
:105D50007A6F050E7B6F980E7F6F580E806F7C8F69
:105D600010D00001CF0E756F050E766F070E786F9D
:105D7000796BC10E776F05D032C4E3F00001778FE5
:105D800000D012000501CF6BC20ED06F010ED16F93
:105D9000D26BD36BD46B080ED56F0001D76B1A0E84
:105DA000E66E010EE66E44EC1DF0E552E5521E0E65
:105DB000E66E020EE66E44EC1DF0E552E552870EEB
:105DC000E66E080EE66E050EE66EE66A020EE66EFA
:105DD000EBEC1DF0146E050EE15E1450F3CFDFF016
:105DE000F4CFE0F00001E16BE26BD86B1200D9CF89
:105DF000E6FFE1CFD9FF0001D76BDF51E01102E1EF
:105E0000000E08D0DFC0E9FFE0C0EAFFEF50800BD2
:105E100001E0010E000945E1FC0EDBCF14F0DFC00C
:105E2000E9FFE0C0EAFFEE52EF50D880145408E2D8
:105E3000DFC0E9FFE0C0EAFFEE52FC0EEFCFDBFF70
:105E4000D76BFC0EDB50D75D19E2D751EA6A080F19
:105E5000E96E050EEA22EF50E66ED751E76EFD0EB1
:105E6000DBCFE9FFFE0EDBCFEAFFE750E926000EAD
:105E7000EA22E552E750EF6ED72BE3D7870EE66EA6
:105E8000080EE66E050EE66EE66A020EE66EEBECB6
:105E90001DF0146E050EE15E1450F3CFDFF0F4CF69
:105EA000E0F00001D75100D0E552E7CFD9FF120052
:105EB000D9CFE6FFE1CFD9FF0001D8510CE1FD0EAB
:105EC000DBCFD9F0FE0EDBCFDAF0FC0EDBCFDDF05E
:105ED000010EDE6FD86FE552E7CFD9FF1200D9CFA0
:105EE000E6FFE1CFD9FF030EE1260001D85101E022
:105EF0002ED0DF6AFD0EDBCF08F0FE0EDBCF09F0FF
:105F0000DE5208C0DEFF09C0DDFFDD52DF2ADF50B0
:105F1000146E156AFF0E141801E1155001E10BD043
:105F2000010EDBCFE9FFDB2A020EDBCFEAFF01E344
:105F3000DB2AEF50EBE1FD0EDBCFD9F0FE0EDBCF1D
:105F4000DAF0DFCFDDF00001010EDE6FD86F030E57
:105F5000E15C02E2E16AE552E16EE552E7CFD9FF8A
:105F60001200D9CFE6FFE1CFD9FF030EE1260001F1
:105F7000D85101E02FD0DF6AFD0EDBCF08F0FE0E16
:105F8000DBCF09F0DE5208C0DEFF09C0DDFFDD52C5
:105F9000DF2ADF50146E156AFF0E141801E1155048
:105FA00001E10CD0010EDBCFF6FFDB2A020EDBCFC6
:105FB000F7FF01E3DB2A0800F550EAE1FD0EDBCF35
:105FC000D9F0FE0EDBCFDAF0DFCFDDF00001DE6BC3
:105FD000010ED86F030EE15C02E2E16AE552E16E68
:105FE000E552E7CFD9FF1200D9CFE6FFE1CFD9FFC5
:105FF000020EE1260001E151E21102E1000E08D09B
:10600000E1C0E9FFE2C0EAFFEF50800B01E0010EC2
:10601000000901E085D0030ED85D01E1D86BD851AD
:1060200001E17ED0020ED85D16E1E66A000EE66E52
:10603000E66A010EE66E020EE66EEBEC1DF0146EE3
:10604000050EE15E1450F3CFE1F0F4CFE2F0000171
:10605000030ED86F65D0D80563E1400E146E156A43
:10606000DD51145C000E155803E2400EDF6E02D0C5
:10607000DDC0DFFFDF50DD5DDD6F8F0EDB6F050EF6
:10608000DC6F010EDFCFDBFFDE5117E1010EDB50CD
:1060900013E0D9C0F6FFDAC0F7FF0800F550DBC007
:1060A000E9FFDCC0EAFFEF6EDB2B000EDC23D92B0F
:1060B000DA23010EDB06EAD715D0010EDB5012E021
:1060C000D9C0E9FFDAC0EAFFEF50DBC0E9FFDCC06E
:1060D000EAFFEF6EDB2B000EDC23D92BDA23010E57
:1060E000DB06EBD7DD5108E1400EDF5C03E1020E79
:1060F000D86F02D0030ED86FDFCFE6FF8F0EE66EAB
:10610000050EE66E010EE66E020EE66EEBEC1DF07D
:10611000146E050EE15E1450F3CFE1F0F4CFE2F01F
:10612000020EE15C02E2E16AE552E16EE552E7CF80
:04613000D9FF120081
:0C613400006A0EAEA3EF30F00D6C0E1EE2
:10614000E86A0E22001E09AEABEF30F0086C091EA3
:10615000E86A0922001EBEEC33F009BEBBEF30F046
:1061600000AE000C086C091EE86A0922046C051ECA
:10617000E86A0522000C00BEB2EF30F00188FF0C87
:10618000006A0EAECBEF30F00C6C0D1E0E1EE86AEE
:106190000D220E22001E09AED5EF30F0076C081E4E
:1061A000091EE86A08220922001E32EC33F009BEFB
:1061B000E8EF30F000AE000C076C081E091EE86A1C
:1061C00008220922036C041E051E04220522000C6D
:1061D00000BEDCEF30F00188FF0C006AE86A0EAE0A
:1061E000FAEF30F00B6C0C1E0D1E0E1E0C220D2251
:1061F0000E22001E09AE05EF31F0066C071E081EC8
:10620000091E072208220922001ECEEC32F009BE28
:106210001CEF31F000AE000C066C071E081E091EB4
:10622000E86A072208220922026C031E041E051ECA
:10623000032204220522000C00BE0CEF31F001887D
:10624000FF0C08C012F008500D02F4CF07F0F3CF96
:1062500006F009500E02F4CF09F0F3CF08F00D025A
:10626000F3500726F4500822E86A092212500E0261
:0E627000F3500726F4500822E86A0922000CB9
:02627E0012010B
:10628000000202000008D8040A0000010102000117
:1062900009024300020100C03209040000010202A9
:1062A0000100052400100104240202052406000157
:1062B000052401000107058103080002090401000B
:1062C000020A0000000705020240000007058202E2
:1062D00040000004030904340369004300690072AC
:1062E00000630075006900740020005400650063BD
:1062F0000068006E006F006C006F00670069006549
:106300000073000000000000000000340369004337
:10631000005000310032002000620079002000505F
:106320000049004300630069007200630075006962
:106330000074002E0063006F006D002000000090CC
:0763400062D362D7620B6318
:086348002A0EF66E100EF76E2E
:10635000000EF86E02010900F550EF6F0900F550CC
:10636000F06F03E1EF6701D03DD00900F550EA6F0F
:106370000900F550EB6F0900F550EC6F09000900BA
:10638000F550E96E0900F550EA6E090009000900B0
:10639000F550ED6F0900F550EE6F09000900F6CFDA
:1063A000F1F2F7CFF2F2F8CFF3F2EAC2F6FFEBC266
:1063B000F7FFECC2F8FF0201ED5302E1EE5307E0F4
:1063C0000900F550EE6EED07F8E2EE07F9D7F1C2DD
:1063D000F6FFF2C2F7FFF3C2F8FF0201EF07000E6B
:0663E000F05BBFD71200C4
:0A63E600D9CFE6FFDACFE6FFFA0E8A
:1063F000E3CFD9FFFB0EE3CFDAFFFC0EE3CFE9FFDB
:10640000FD0EE3CFEAFFE9CFF3FFEACFF4FFF80E8A
:10641000E35003E1F90EE35008E0F80EE30602E270
:10642000F90EE306DECFEEFFF2D7FF0EE3CFDAFF81
:10643000E552FF0EE3CFD9FFE5521200FE0EE3CF87
:10644000E9FFFF0EE3CFEAFFE9CFF3FFEACFF4FF66
:10645000FB0EE35003E1FC0EE35009E0FB0EE30604
:1064600002E2FC0EE306FD0EE350EE6EF1D71200E1
:1064700006500B02F3CF02F0F4CF03F00C02F350FE
:106480000326000EF420046E06500D02F35004267D
:10649000000EF420056E06500E02F350052607503C
:1064A0000B02F3500326F4500422000E052207507D
:1064B0000C02F3500426F450052207500D02F3504D
:1064C000052608500B02F3500426F450052208500C
:1064D0000C02F350052609500B02F350052612005A
:1064E000D9CFE6FFDACFE6FFE1CFD9FFE2CFDAFF7F
:1064F000E652E652FC0EDBCF14F0FD0EDBCF15F0BA
:10650000060ED89014361536E804FBE114C0DEFF01
:1065100015C0DDFF010EDB50BB6EDF50E840E840E8
:106520003F0B300B146ECF0EBA141410BA6EE55236
:0E653000E552E552E5CFDAFFE7CFD9FF1200C2
:02653E00D9CFB3
:10654000E6FFDACFE6FFE1CFD9FFE2CFDAFFE6528E
:10655000E652FC0EDBCF14F0FD0EDBCF15F0060E7D
:10656000D89014361536E804FBE114C0DEFF15C0E0
:10657000DDFF010EDB50BE6EDF50E840E8403F0B10
:10658000300B146ECF0EBD141410BD6EE552E552E3
:0C659000E552E5CFDAFFE7CFD9FF12009B
:04659C00056A046A1E
:1065A000036A026A200EE76ED89006360736083670
:1065B000093602360336043605360B50025C0C50A1
:1065C00003580D5004580E50055809E30B50025E55
:1065D0000C50035A0D50045A0E50055A062AE72E45
:0465E000E4D71200EA
:0C65E400D9CFE6FFDACFE6FFE1CFD9FF08
:1065F000E2CFDAFFFD0EDB507E0BCD6EFD0EDBAC85
:1066000002D0CD8E01D0CD9ECF6ACE6A9E90DBAEF9
:1066100002D09D8001D09D90CD80E552E5CFDAFF7C
:06662000E7CFD9FF1200D4
:0A662600D9CFE6FFDACFE6FFE1CF9F
:10663000D9FFE2CFDAFFE652E652D650DF6E010E06
:10664000D7CFDBFFDECF14F0DDCF15F014C0F3FFA2
:1066500015C0F4FFE552E552E552E5CFDAFFE7CF8A
:04666000D9FF12004C
:0C666400056A046A036A180EE76ED890FD
:106670000736083609360336043605360C50035CF7
:106680000D5004580E50055807E30C50035E0D5092
:0E669000045A0E50055A072AE72EEAD71200C8
:02669E00D9CF52
:1066A000E6FFDACFE6FFE1CFD9FFE2CFDAFFE6522D
:1066B000E652FC0EDBCFDEFFDBCFDDFF010EDB5051
:1066C000CF6EDF50CE6EE552E552E552E5CFDAFFF0
:0666D000E7CFD9FF120024
:0A66D600D9CFE6FFDACFE6FFE1CFEF
:1066E000D9FFE2CFDAFFE652E652FC0EDBCFDEFF47
:1066F000DBCFDDFF010EDB50D76EDF50D66EE552EB
:0E670000E552E552E5CFDAFFE7CFD9FF1200F0
:02670E00D9CFE1
:10671000E6FFDACFE6FFE1CFD9FFE2CFDAFFFD0EE9
:10672000DB507F0BD56ED76AD66AF294FD0EDBAED6
:1067300002D0F28A01D0F29AD58EE552E5CFDAFF87
:06674000E7CFD9FF1200B3
:0A674600D9CFE6FFDACFE6FFE1CF7E
:10675000D9FFE2CFDAFFFD0EDB50FB0BCA6ECC6A2D
:106760009E92FD0EDBAE02D09D8201D09D92CA8426
:0C677000E552E5CFDAFFE7CFD9FF1200B9
:04677C00056A046A3C
:10678000100EE76ED89008360936043605360D50DF
:10679000045C0E50055805E30D50045E0E50055A7A
:0867A000082AE72EF0D71200D1
:0867A800000EF36E00EE00F09C
:1067B000080E01D81200EA6002D0EE6AFCD7F3504E
:0867C000E9601200EE6AFCD74B
:0867C80013EE00F023EE00F0D7
:1067D000F86A019CA4EC31F0F8EC33F0CDEC2BF02E
:0467E000FBD71200D1
:0667E400CD909D90120013
:0667EA00D59EF29A120098
:0267F000120095
:0E67F200000000000000000000000000000099
:106800000000000000000000000000000000000088
:106810000000000000000000000000000000000078
:016820000077
:020000040030CA
:0100000024DB
:010001000EF0
:010002003FBE
:010003001EDE
:010005008179
:010006008178
:010008000FE8
:01000900C036
:01000A000FE6
:01000B00E014
:01000C000FE4
:01000D0040B2
:00000001FF
